:1000000000400020B1440000F1440000F34400002F
:1000100000000000000000000000000000000000E0
:10002000000000000000000000000000F544000097
:100030000000000000000000F7440000F944000048
:10004000FB440000FB440000E54C0000FB440000C2
:10005000FB44000000000000FB440000FB440000E3
:10006000FB44000029470000FB440000FB44000063
:10007000FB440000FB440000FB440000FB44000084
:10008000FB440000894D0000FB440000FB440000DD
:10009000FB440000FB440000FB440000FB44000064
:1000A000FB440000FB4400000000000000000000D2
:1000B0000000000000000000000000000000000040
:1000C000054B0648033310B51B1A062B03D9044B06
:1000D000002B00D0984710BD780100207801002047
:1000E000000000000648074910B5091A8910CB0F17
:1000F0005918491003D0044B002B00D0984710BD6D
:1001000078010020780100200000000010B5074CA5
:100110002378002B09D1FFF7D3FF054B002B02D02A
:10012000044800E000BF0123237010BD78010020C7
:1001300000000000A8730000094B10B5002B03D08D
:100140000849094800E000BF08480368002B02D1B5
:10015000FFF7C8FF10BD064B002BF9D09847F7E713
:10016000000000007C010020A87300007401002042
:1001700000000000164B002B00D1144B9D4640227E
:1001800092029A1A924600218B460F461348144A4F
:10019000121A05F068F80F4B002B00D098470E4B51
:1001A000002B00D098470020002104000D000D48CE
:1001B000002802D00C4800E000BF05F011F8200034
:1001C000290004F0A7FD04F0E5FFC0460000080088
:1001D0000040002000000000000000007801002026
:1001E0000420002000000000000000000123034064
:1001F0000200181E04D1042A03D91068000900E087
:100200000020704710B50400FFF7F0FF0300002046
:1002100083420BD0013B9B00181DE2181279002A83
:1002200003D001338342F8D100E0180010BD012251
:10023000016810B5114201D0002903DA102000F046
:10024000E3F903E04910062001F004FF10BD016846
:1002500010B5CB0701D5002903DA102000F0D4F93E
:1002600006E04910033189100022052001F0F2FE5A
:1002700010BD70B50568AB0728D1042D26D90F2312
:100280002A6846681340062B09D12800FFF7AEFF05
:10029000012383421DDC9A00AE500133F9E7052BA0
:1002A00014D1F30703D4132000F0AEF912E0761056
:1002B000FF2EF8D82800FFF799FF2C1D230080009F
:1002C0002018984205D91E700133FAE70B2000F080
:1002D0009BF9002070BD70B50468E30701D41120BC
:1002E0002DE04568AB0729D1042D27D90F262B68AF
:1002F00064101E40062E0BD1002C04DD2800FFF7F1
:1003000075FF844201DD122019E0A400605918E055
:10031000331F012B12D82800FFF768FF8000042E3E
:1003200002D12800FFF76EFF002CECDDA042EADBD3
:1003300001232C19E0784000184302E00B2000F064
:1003400063F970BDF8B5012304681C4201D1112086
:100350002FE00325466835402AD1042E28D90F23E3
:100360003268641087681340062B0BD1002C04DD23
:100370003000FFF73BFF844201DD122019E0A400AA
:10038000A75113E0052B13D1002CF6DD3000FFF749
:100390002DFF80008442F0DC01231F4201D1132095
:1003A00007E07F10FF2FFAD83419E770280002E029
:1003B0000B2000F029F9F8BD006810B5830717D1AC
:1003C000042815D90F2302681340062B02D1FFF72A
:1003D0000DFF0BE0052B05D1FFF708FFC00001233F
:1003E000184308E0042B03D1FFF70CFF4000F6E7A9
:1003F0000B2000F009F910BD10B50324006804407B
:1004000006D1042804D90F2302681340042B01D01D
:100410000E2011E001F05AFE0378233B5942594166
:1004200010224018210005F0F7FB80239B05C2181D
:10043000054B9A4203D9142000F0E6F802E00123AC
:100440004000184310BDC046FFFFFF3F10B5012418
:100450000368234202D04268224203D10D2000F0FB
:10046000D3F808E004495B1052101B070A401343FD
:1004700018684000204310BDFCFFFF0F01210368F6
:1004800010B50B4205D042680A4202D0806808428B
:1004900003D10D2000F0B8F808E005495B105210B8
:1004A0001B070A40401013431860002010BDC046CF
:1004B000FCFFFF0F012303400200181E01D0501063
:1004C00002E00D22014B1A707047C04694010020D3
:1004D000012303400200181E04D1042A03D9106826
:1004E000000900E00020704770B50D000400FFF720
:1004F000EFFF86002800FFF7EBFF830000209E42FD
:100500000ED1231D9E1904351A009E4207D9297861
:100510001278013301358A42F6D0002000E0012034
:1005200070BD0000F0B585B00393019002912D4E8F
:100530002D4B002A02D002223270013A00251A60A7
:100540001B68F554019B9D424ADA029AAB00D058D1
:10055000254B1C68C8239B0037191C1B012318421C
:1005600002D04310214A1FE0214A002802D004286B
:1005700005D1204A2100380005F03CFA18E0042893
:1005800010D90F2302681340042B04D101F09EFD03
:10059000194A030008E0062B05D1FFF799FF174A17
:1005A000030001E00123164A2100380005F022FA79
:1005B000300005F085FA039B0B4A002B01D1106037
:1005C0000CE0019B013B9D42F9DA0E4B9842F6DCB0
:1005D000431C1360202232540022F2540135B1E74B
:1005E00005B0F0BDA00100209C010020E5690000DD
:1005F000B8690000BE6900002C6C0000C3690000EF
:10060000D46900001F030000014B187000207047E0
:100610009401002070B502F023FE094C0100251D55
:100620001F22280005F053FA280005F049FA042398
:1006300004308008000118432060200070BDC046CF
:10064000C0040020C368F0B59D00836887B05D19C1
:10065000030018330393036902909F00039BDF1983
:1006600043699E000093039B9E19D24B1B78002B7D
:100670000FD17F222B68D0491C1213409B005B587E
:1006800000960435019235E0CA4B1B78002B29D027
:10069000009E029BC74C9B6821780093EA1A029B3C
:1006A00092109B7812021A43029B587802F064FB66
:1006B0000023029A2370137000960497029B039AFA
:1006C0009B68ED1A0193029BAD10DD60049B9F1A9D
:1006D000029BBF101F61009B9B1A029A9B105361E3
:1006E00001F005FC2B68019A1C121340B24A9B00D2
:1006F0009B5804359F46029B587802F035FB002337
:10070000029A1370D9E7039B3A1DD11AA94B8B2982
:1007100003DD1A22009E1A70BBE71B783C60002B99
:1007200002D0009E1700B4E72B6801991C120B4001
:10073000A1499B005B5817000435DBE7039B3A1D7A
:10074000D11A9C4B8B2903DD1A22009E1A70A0E758
:1007500028681B78291D3860002B03D0009E1700E5
:100760000D0096E76B6801991C120B4092499B00A3
:100770005B5817000835BDE7039B3A1DD11A8D4B16
:100780008B2903DD1A22009E1A7082E7A4001B78D1
:100790002C193C60002B02D0009E170079E72B68D3
:1007A00001991C120B4084499B005B5817000435CB
:1007B000A0E7039B3A1DD11A7E4B8B2903DD1A2239
:1007C000009E1A7065E77D48A40021581B783960A7
:1007D000002B02D0009E17005BE72B6801991C12CA
:1007E0000B4075499B005B581700043582E7043FB6
:1007F000724B3A68A400E2506E4B1B78002B01D07C
:10080000009E46E72B68019A1C1213406A4A9B001F
:100810009B5804356EE7694BA600F058FFF74AFE77
:10082000043F04003868FFF745FE24180120634B9D
:1008300064000443F4505F4B1B78002B01D0009EF2
:1008400027E72B68019A1C1213405B4A9B009B58B8
:1008500004354FE7039B3A1DD11A564B8B2903DD14
:100860001A22009E1A7014E70098039C0121A042EE
:1008700002D901000C3909681B783960002B02D0BD
:10088000009E170005E72B6801991C120B404A498E
:100890009B005B58170004352CE7039B3A1DD11AC7
:1008A000444B8B2903DD1A22009E1A70F1E6009951
:1008B000039881420AD90B000C3B1B6840495B102E
:1008C0006418E41A009BA400E35802E01821197090
:1008D00000233B60374B1B78002B02D0009E170093
:1008E000D7E62B6801991C120B4033499B005B58DB
:1008F00017000435FEE6009B039A93420BD90C3B8C
:1009000019682F4B043FE3184910591A3A68009BA5
:100910008900CA5002E01822264B1A70254B1B781A
:10092000002B01D0009EB4E62B68019A1C121340E4
:10093000214A9B009B580435DCE6009B039A9342B6
:100940001CD9009E1E4B0C3EE4183368009A5B10C5
:10095000E31A9B009858FFF7ADFD043F04903868F8
:10096000FFF7A8FD3168049B4910611A012418188B
:100970004000009B89002043C85002E018220D4B24
:100980001A700C4B1B78002B01D0009E81E62B685F
:10099000019A1C121340084A9B009B580435A9E693
:1009A000039B3A1DD11A034B8B290BDD1A22009EA3
:1009B0001A706EE694010020B8670000E41E002063
:1009C000FDFFFF3F0099A40061581B783960002BA0
:1009D00002D0009E17005CE62B6801991C120B40A8
:1009E000CF499B005B581700043583E6043F009B0A
:1009F0003A68A400E250CB4B1B78002B01D0009E3C
:100A000047E62B68019A1C121340C54A9B009B586D
:100A100004356FE6009BA4001C192368043F386866
:100A20005E10FFF747FD36180120BE4B76001B789D
:100A300006432660002B01D0009E2AE62B68019A0F
:100A40001C121340B64A9B009B58043552E6039B88
:100A5000A4003F1BB34CBB420DD82378002B01D020
:100A6000009E16E62B68019A1C121340AC4A9B00AC
:100A70009B5804353EE6AC4801F09EFA2378002BE3
:100A800001D0009E05E62B68019A1C121340A44A6F
:100A90009B009B5804352DE6A300ED18002C00DACE
:100AA0000BE6A04B1B78002B01D0009EF1E52B68D4
:100AB000019A1C1213409A4A9B009B58043519E670
:100AC0003B1F04931B680593042B04D1A300ED186E
:100AD000002C00DAF2E5934B1B78002B02D0009E2D
:100AE000049FD6E52B68019A1C1213408C4A9B0088
:100AF0009B58049F0435FDE53B1F04931B68059339
:100B0000002B04D1A300ED18002C00DAD6E5854BAC
:100B10001B78002B02D0009E049FBAE52B68019A37
:100B20001C1213407E4A9B009B58049F0435E1E54C
:100B30003A1F13685B10013B002B07DD01215B00AE
:100B4000A4000B4304972D191360B7E5754B1700EC
:100B50001B78002B01D0009E9BE52B68019A1C128C
:100B600013406F4A9B009B580435C3E53A00039B32
:100B70000C32D31A8B2B04DD1A226A4B009E1A709A
:100B800087E5FF2361005B000B4001210B433B60C5
:100B9000029B03989B6824120493ED1A029BAD10EC
:100BA0009B782D021D43009B8D401B1A9B108B4090
:100BB0000B43BB60029B0D437D609C70E4B25B4BBA
:100BC000E4000299E35816008B6056490978002921
:100BD00003D008331D0017005BE51D0001999B68D9
:100BE0000C351C120B404E499B005B5800921700BD
:100BF00080E53B1F1E68039A009B93422AD104970D
:100C00000A20F30716D4B3070DD1042E0BD90F23F6
:100C100032681340042B06D1300001F057FA04F07B
:100C20004FFF063006E00720042E03D0002E01D02F
:100C300080208000643001F063FE002801D1043D73
:100C40003CE5029B3100587802F0A8F80023029A94
:100C5000137033E5009B009A0C3B1B6802995B10F4
:100C60009B005B421F00D3180C3B1E601300083B27
:100C70001B68083FD7195A108A70D2B22B49D2008C
:100C80005B0055589B0A029A9B009560ED18009BEB
:100C9000043B1E68039B7610B6009E19214B1B78FF
:100CA000002B00D0F5E42B68019A1C1213401C4A5B
:100CB0009B009B58009604351CE53B1F1868FFF706
:100CC000F9FBA40006003F1B1E2833DC00280EDCC5
:100CD000144B1B78002B01D0009EDAE42B68019A9C
:100CE0001C1213400E4A9B009B58043502E502F08B
:100CF0009DFA033E361802F099FA0D4B801B98427C
:100D0000F9D8084B1B78002B01D0009EC1E42B685A
:100D1000019A1C121340024A9B009B580435E9E4D7
:100D2000B867000094010020E8690000EC1600207C
:100D30009F8601000123029A137002F077FA029B4A
:100D40000A3886195E60B8E43B1F1868FFF7B2FBEB
:100D5000A40004903F1B00280EDCCF4B1B78002B17
:100D600001D0009E95E42B68019A1C121340CB4AD7
:100D70009B009B580435BDE4C94B049A009E9A42DF
:100D800003DD1D22C44B1A7083E40123029A137001
:100D900002F04CFAFA23049A9B005343029A0A3B4E
:100DA0001B18536089E4A300FF1A002320001A00D7
:100DB0003900FFF7B7FBBB4EBB4C3168200001F098
:100DC00039FF3168200001F0F0FFB34B1B78002B96
:100DD00001D0009E5DE42B68019A1C121340AF4ABB
:100DE0009B009B58043585E4AB4BA4001B783F1B4C
:100DF000002B01D0009E4CE42B68019A1C1213407A
:100E0000A64A9B009B58043574E401F0BFFD01F035
:100E10006EF83B1F1868002823D1083B1868C307E9
:100E200001D5401016E083070FD104280DD90F23F8
:100E300002681340062B02D1FFF74AFB0AE0052B9C
:100E400003D1FFF745FB800004E01922924B009E7E
:100E50001A701EE43A0001214300083A0B43136064
:100E600001E040100138002832DD01224300134325
:100E7000391F0B603B00083B1B681341181A3B00ED
:100E80000C3B1B68134203D08018A400904015E06F
:100E9000990717D1042B15D90F211E683140062957
:100EA00006D101308000C358009AA400A35010E07E
:100EB000052907D118180079A4004000009B1043B1
:100EC000E05006E01922744B009E1A70FFF7E1FB18
:100ED0000435714B1B78002B02D0009EFFF7D9FB25
:100EE0002B68019A1C1213406C4A9B009B580435D6
:100EF000FFF700FCA300039AFB189B1A8B2B01DC65
:100F0000002205E01A22644B009E1A70FFF7C1FB15
:100F1000631E002C03DD3A601C000437F8E75E4BCB
:100F20001B78002B02D0009EFFF7B3FB2B68019AC1
:100F30001C121340594A9B009B580435FFF7DAFBFB
:100F4000A3009C46F81A002C04DC1C22524B0026FD
:100F50001A7015E0002103685B1001268A00825890
:100F6000164003D10D224C4B1A7009E052109342E7
:100F700000DD130001318C42EFDC01265B001E43D3
:100F80006346FF1A444B06601B780437002B02D0DF
:100F9000009EFFF77EFB2B68019A1C1213403F4A0C
:100FA0009B009B580435FFF7A5FBA3009C46F81A4D
:100FB000002C04DC1C22384B00261A7015E000219E
:100FC00003685B1001268A008258164003D10D2267
:100FD000314B1A7009E05210934200DA13000131CC
:100FE0008C42EFDC01265B001E436346FF1A2A4B4E
:100FF00006601B780437002B02D0009EFFF749FBE8
:101000002B68019A1C121340244A9B009B580435FC
:10101000FFF770FB3B00083B1868FFF74BFA3B1FDC
:1010200004901868FFF746FA049AA600BC1B002338
:10103000824200DA04332360174BBF1B1B7804374E
:10104000002B02D0009EFFF724FB2B68019A1C1294
:101050001340124A9B009B580435FFF74BFBA3003B
:10106000FE1A04933B00083B1868FFF723FA3B1F66
:1010700004001868FFF71EFAE20FC317A04253419D
:101080009B003360049BFF1A034B04371B78002B33
:101090000CD0009EFFF7FDFA94010020B867000015
:1010A00080EE36009C010020A00100202B68019AF0
:1010B0001C121340D84A9B009B580435FFF71AFBBB
:1010C0003B00083B18683B1F1968A300884202D107
:1010D000FB1A042222E004281ED90122104201D06A
:1010E000114219D10326304215D10F2302681A404C
:1010F000042A10D131420ED104290CD90A681340B8
:10110000042B08D1FFF7F0F9431E9841A600BE1B3F
:101110008000306003E0A3000022FB1A1A60BF4B7E
:10112000A4001B783F1B0437002B02D0009EFFF762
:10113000B0FA2B68019A1C121340B74A9B009B58C7
:101140000435FFF7D7FA3B00083B18683B1F1968C6
:10115000A300884202D1FB1A002223E004281FD9F1
:101160000122104201D011421AD10326304216D179
:101170000F2302681A40042A11D131420FD10429E9
:101180000DD90A681340042B09D1FFF7ADF903000C
:1011900058425841A600BE1B8000306003E0A30007
:1011A0000422FB1A1A609D4BA4001B783F1B0437D6
:1011B000002B02D0009EFFF76CFA2B68019A1C12DC
:1011C0001340954A9B009B580435FFF793FAA30000
:1011D000FE1A04933B00083B1868FFF76BF93B1FAE
:1011E00004001868FFF766F9E217C30F8442534101
:1011F0009B003360049BFF1A884B04371B78002B3D
:1012000002D0009EFFF745FA2B68019A1C1213408A
:10121000814A9B009B580435FFF76CFA3B00083B62
:101220001868FFF747F93B1F04901868FFF742F969
:10123000049AA600BC1B0023824200DD0433236015
:10124000764BBF1B1B780437002B02D0009EFFF7A4
:1012500020FA2B68019A1C1213406F4A9B009B587E
:101260000435FFF747FA3B1F1B686C4AA400042BA8
:1012700002D13B1B002103E0002B03D104213B1BC7
:10128000196001E00C23137013783F1B0437002B07
:1012900002D0009EFFF7FDF92B68019A1C12134043
:1012A0005D4A9B009B580435FFF724FAA300FC1A03
:1012B00004933B00083B1868FFF7FCF83B1F06004F
:1012C0001868FFF7F7F836180120049B7600FF1A1C
:1012D000524B06431B7826600437002B02D0009E39
:1012E000FFF7D7F92B68019A1C1213404A4A9B005A
:1012F0009B580435FFF7FEF9A300FE1A04933B0048
:10130000083B1868FFF7D6F83B1F04001868FFF782
:10131000D1F8241A0120049B6400FF1A3F4B0443B8
:101320001B7834600437002B02D0009EFFF7B1F920
:101330002B68019A1C121340374A9B009B580435B6
:10134000FFF7D8F9A300FC1A04933B00083B186888
:10135000FFF7B0F83B1F06001868FFF7ABF84643ED
:101360000120049B7600FF1A2C4B06431B78266055
:101370000437002B02D0009EFFF78BF92B68019AEF
:101380001C121340244A9B009B580435FFF7B2F906
:101390003B00083B1868FFF78DF83B1F0490186866
:1013A000FFF788F80100049803F0BCFD0123A400B6
:1013B0003E1B370040001843184B30601B78043741
:1013C000002B02D0009EFFF764F92B68019A1C12D3
:1013D0001340114A9B009B580435FFF78BF93B00E3
:1013E000083B1868FFF766F83B1F04901868FFF782
:1013F00061F80100049803F07BFE0123A4003E1B6A
:10140000370049001943054B31601B780437002B26
:1014100006D0009EFFF73DF9B86700009401002058
:101420002B68019A1C121340E74A9B009B58043515
:10143000FFF760F93B1F1868FFF73CF8C317C018A7
:101440005840012340001843E04BA4001B783E1B8A
:101450003060371D002B02D0009EFFF71AF92B6871
:10146000019A1C121340D84A9B009B580435FFF781
:1014700041F9A300FE1A05933068012C03D1FFF750
:1014800019F8049008E0FFF715F804007068FFF7FA
:1014900011F80130031B0493049B002B01DC012392
:1014A000049304F059FA049903F022FE0C19012167
:1014B000059B6400FF1AC54B0C431B78346004374E
:1014C000002B02D0009EFFF7E4F82B68019A1C1253
:1014D0001340BD4A9B009B580435FFF70BF9A4004D
:1014E0003E1B3000FEF788FFB84B30601B78371D7D
:1014F000002B02D0009EFFF7CCF82B68019A1C123B
:101500001340B14A9B009B580435FFF7F3F8A30042
:10151000FE1A04933B00083B1868FEF7CBFF3B1F05
:1015200004001868FEF7C6FF04400120049B640015
:10153000FF1AA64B04431B7834600437002B02D0FB
:10154000009EFFF7A6F82B68019A1C1213409E4AD2
:101550009B009B580435FFF7CDF8A300FC1A0493B9
:101560003B00083B1868FEF7A5FF3B1F0600186804
:10157000FEF7A0FF06430120049B7600FF1A934B61
:1015800006431B7826600437002B02D0009EFFF72D
:1015900080F82B68019A1C1213408B4A9B009B58C1
:1015A0000435FFF7A7F8A300FC1A04933B00083B9F
:1015B0001868FEF77FFF3B1F06001868FEF77AFFEA
:1015C00046400120049B7600FF1A804B06431B789F
:1015D00026600437002B02D0009EFFF75AF82B68D4
:1015E000019A1C121340784A9B009B580435FFF760
:1015F00081F83B1F1868FEF75DFFC04301234000E0
:101600001843724BA4001B783E1B3060371D002B23
:1016100002D0009EFFF73DF82B68019A1C12134080
:10162000694A9B009B580435FFF764F8A300FE1A33
:1016300004933B00083B1868FEF73CFF3B1F040087
:101640001868FEF737FF8440012364001C43049BA5
:101650003460FF1A5D4B04371B78002B02D0009ECC
:10166000FFF717F82B68019A1C121340564A9B008B
:101670009B580435FFF73EF8A300FE1A04933B0085
:10168000083B1868FEF716FF3B1F04001868FEF7BA
:1016900011FF0441012364001C43049B3460FF1AC2
:1016A0004A4B04371B78002B02D0009EFEF7F1FF57
:1016B0002B68019A1C121340434A9B009B58043527
:1016C000FFF718F8A4003E1B3000FEF7B0FD3F4BBB
:1016D00030601B78371D002B02D0009EFEF7D9FF2B
:1016E0002B68019A1C121340374A9B009B58043503
:1016F000FFF700F8A4003E1B3000FEF7A8FD334BB7
:1017000030601B78371D002B02D0009EFEF7C1FF12
:101710002B68019A1C1213402B4A9B009B580435DE
:10172000FEF7E8FFA4003F1B3800FEF7A2FD274BA1
:101730001B78002B02D0009EFEF7ABFF2B68019AAE
:101740001C121340204A9B009B580435FEF7D2FF21
:10175000A4003E1B3000FEF7BEFD1C4B30601B7822
:10176000371D002B02D0009EFEF793FF2B68019AD5
:101770001C121340144A9B009B580435FEF7BAFF15
:10178000A4003F1B3800FEF7DDFD104B1B78002B3B
:1017900002D0009EFEF77DFF2B68019A1C121340B9
:1017A000094A9B009B580435FEF7A4FFA4003E1B8A
:1017B0003000FEF701FE054B30601B78371D002B13
:1017C00006D0009EFEF765FFB86700009401002078
:1017D0002B68019A1C121340E64A9B009B58043563
:1017E000FEF788FF039A3B1D0493E34C9B1A8B2B57
:1017F00004DD1A23009E2370FEF74BFF01F020FD4D
:1018000001234000184323783860002B03D0009E4A
:10181000049FFEF73EFF2B68019A1C121340D54A25
:101820009B009B58049F0435FEF764FF039A3B1D01
:101830000493D14C9B1A8B2B04DD1A23009E23703A
:10184000FEF727FF01F0F2FCCC4B400018400123CB
:10185000184323783860002B03D0009E049FFEF7C6
:1018600018FF2B68019A1C121340C24A9B009B5818
:10187000049F0435FEF73EFFA4003E1B3000FEF738
:10188000E5FDBD4B30601B78371D002B02D0009E5C
:10189000FEF7FFFE2B68019A1C121340B54A9B000D
:1018A0009B580435FEF726FFA4003F1B3800FEF7C7
:1018B000E5FDB14B1B78002B02D0009EFEF7E9FE40
:1018C0002B68019A1C121340AA4A9B009B580435AE
:1018D000FEF710FFA300FB1A0493012320001A0057
:1018E0000499FEF71FFEA64C2068643001F008F84A
:1018F000002816D0029B21685A78A24801F063FAAA
:1019000015E0A300FB1A0493200001230022049990
:10191000FEF708FE9A4C2068643000F0F1FF0028C2
:1019200002D1043DFEF7C9FE964801F003F90123F8
:10193000029A137001F07AFC962223685200063353
:1019400053431818029B5860FEF7B8FEFEF762FE7C
:10195000894BA4001B783E1B3060371D002B02D042
:10196000009EFEF796FE2B68019A1C121340814AD6
:101970009B009B580435FEF7BDFEA4003E1B3000C3
:1019800001F092FC7C4B30601B78371D002B02D09D
:10199000009EFEF77EFE2B68019A1C121340754ACA
:1019A0009B009B580435FEF7A5FEA4003E1B3000AB
:1019B00001F07CFC704B30601B78371D002B02D08F
:1019C000009EFEF766FE2B68019A1C121340694ABE
:1019D0009B009B580435FEF78DFEA4003E1B300093
:1019E00001F066FC644B30601B78371D002B02D081
:1019F000009EFEF74EFE2B68019A1C1213405D4AB2
:101A00009B009B580435FEF775FEA4003F1B380071
:101A100001F06CFC584B1B78002B02D0009EFEF7A7
:101A200038FE2B68019A1C121340524A9B009B58A7
:101A30000435FEF75FFEA4003E1B300001F078FC89
:101A40004D4B30601B78371D002B02D0009EFEF7F7
:101A500020FE2B68019A1C121340464A9B009B589B
:101A60000435FEF747FEA4003F1B380001F092FC4E
:101A7000414B1B78002B02D0009EFEF70AFE2B681C
:101A8000019A1C1213403B4A9B009B580435FEF7F9
:101A900031FE0121200001F065FC374B1B78002B43
:101AA00002D0009EFEF7F5FD2B68019A1C12134030
:101AB000304A9B009B580435FEF71CFE0021200095
:101AC00001F050FC2C4B1B78002B02D0009EFEF73F
:101AD000E0FD2B68019A1C121340264A9B009B587C
:101AE0000435FEF707FEA4003E1B300001F070FC39
:101AF000214B30601B78371D002B02D0009EFEF773
:101B0000C8FD2B68019A1C1213401A4A9B009B586F
:101B10000435FEF7EFFDA4003E1B300001F06CFC25
:101B2000154B30601B78371D002B02D0009EFEF74E
:101B3000B0FD2B68019A1C1213400E4A9B009B5863
:101B40000435FEF7D7FDA4003F1B380001F02EFC42
:101B5000094B1B78002B02D0009EFEF79AFD2B68E4
:101B6000019A1C121340034A9B009B580435FEF750
:101B7000C1FDC046B867000094010020FEFFFF7F52
:101B80009C010020A0010020A4003F1B380002F0AF
:101B900053F9D84B1B78002B02D0009EFEF779FD3D
:101BA0002B68019A1C121340D34A9B009B580435A2
:101BB000FEF7A0FDA4003E1B300002F08FF9CD4BD4
:101BC00030601B78371D002B02D0009EFEF761FDB0
:101BD0002B68019A1C121340C74A9B009B5804357E
:101BE000FEF788FDA4003F1B380002F0D1F8C14B7E
:101BF0001B78002B02D0009EFEF74BFD2B68019A4C
:101C00001C121340BC4A9B009B580435FEF772FD22
:101C1000A4003E1B300002F0D1F8B64B30601B78B8
:101C2000371D002B02D0009EFEF733FD2B68019A72
:101C30001C121340B04A9B009B580435FEF75AFD16
:101C4000A4003F1B380001F0C7FEAA4B1B78002BF5
:101C500002D0009EFEF71DFD2B68019A1C12134056
:101C6000A54A9B009B580435FEF744FDA4003F1B8A
:101C7000380001F0C7FE9F4B1B78002B02D0009E5E
:101C8000FEF707FD2B68019A1C1213409A4A9B002D
:101C90009B580435FEF72EFDA4003F1B380001F0D1
:101CA000C1FE944B1B78002B02D0009EFEF7F1FC86
:101CB0002B68019A1C1213408F4A9B009B580435D5
:101CC000FEF718FDA4003F1B380001F0D3FE894B3E
:101CD0001B78002B02D0009EFEF7DBFC2B68019ADC
:101CE0001C121340844A9B009B580435FEF702FDEA
:101CF000A300FE1A31002000049302F079F9049B3E
:101D00003060FF1A7B4B04371B78002B02D0009EFB
:101D1000FEF7BFFC2B68019A1C121340764A9B0009
:101D20009B580435FEF7E6FCA300FE1A31002000A4
:101D3000049302F065F9049B3060FF1A6D4B043781
:101D40001B78002B02D0009EFEF7A3FC2B68019AA3
:101D50001C121340684A9B009B580435FEF7CAFCCE
:101D6000A300FE1A31002000049302F051F9049BF5
:101D70003060FF1A5F4B04371B78002B02D0009EA7
:101D8000FEF787FC2B68019A1C1213405A4A9B00ED
:101D90009B580435FEF7AEFCA300FE1A310020006C
:101DA000049301F0C1FF049B3060FF1A514B0437CC
:101DB0001B78002B02D0009EFEF76BFC2B68019A6B
:101DC0001C1213404C4A9B009B580435FEF792FCB2
:101DD000A4003F1B380001F075FE464B1B78002B1A
:101DE00002D0009EFEF755FC2B68019A1C1213408E
:101DF000414A9B009B580435FEF77CFCA300FF1A68
:101E00003900200001F010FF3A4B1B78002B02D064
:101E1000009EFEF73EFC2B68019A1C121340364AC6
:101E20009B009B580435FEF765FCA4003E1B300068
:101E300001F0C6FE2F4B30601B78371D002B02D0FF
:101E4000009EFEF726FC2B68019A1C1213402A4ABA
:101E50009B009B580435FEF74DFCA300FF1A390088
:101E6000200001F08FFE234B1B78002B02D0009E38
:101E7000FEF70FFC2B68019A1C1213401E4A9B00B0
:101E80009B580435FEF736FCA300FF1A39002000EA
:101E900000F0BCFC174B1B78002B02D0009EFEF715
:101EA000F8FB2B68019A1C121340134A9B009B58A5
:101EB0000435FEF71FFCA300FE1A31002000049336
:101EC00000F0A4FC049B3060FF1A0A4B04371B7817
:101ED000002B02D0009EFEF7DCFB2B68019A1C123F
:101EE0001340054A9B009B580435FEF703FC07B0DE
:101EF000F0BDC04694010020B86700000023F7B58C
:101F00005A1E0192002B07DA01F012FC00F0CCFE01
:101F100000F07EFF6423019300263000194B1968FE
:101F20008E4201DB019BEBE7174B1A6801329142AD
:101F300000DC0022A0241A601D68144F6C43E35D8E
:101F4000002B1DD0E419022B16D0012B0ED1002836
:101F500001D101F06BF9A0226A430C4B0C499B188C
:101F60005B68C31A8B4201D80223BB54A0235D4394
:101F7000064BEB5C022B03D12000FEF763FBD1E79D
:101F80000136CBE79801002000000020AC100020B3
:101F90009F860100054B01211A68054B1A6000233A
:101FA000044AD1500433642BFBD17047EC04002069
:101FB000E4040020E41E002000B59BB002000549A7
:101FC00001A803F049FD01A800F0B4FD00F020FFD6
:101FD000FCE7C046F869000037B5174D04002868D3
:101FE000002801D003F02CF9A400200003F01EF912
:101FF0002860002801D1114809E001AB984208D2BD
:102000000F4B02196B440193934202D20D48FFF724
:10201000D3FF042802D808302860083C2B680A4AFD
:102020001C191360094B01211C600023084AD15080
:102030000433642BFBD137BDEC040020096A000097
:102040001CFCFFFF396A0000E4040020E8040020C3
:10205000E41E002070B50D4D0D4E2B684C1CA400E5
:1020600036681C19B44203D90A20FEF7CDFA0BE0FA
:102070002C601D00AC4201D904C5FBE70F22090109
:10208000104008431860180070BDC046E4040020EA
:10209000E80400200322CB1C70B50C00D9171140B6
:1020A000C9180500891000220420FFF7D3FF002380
:1020B000A34204DAE95CC21811710133F8E7E14385
:1020C0000023C917214041180B7170BD10B583075B
:1020D00006D1042804D90F2304C81340042B03D0CD
:1020E0000E20FEF791FA014810BDC046406B00007B
:1020F00030B502248025094B094AED009C505C59FB
:10210000002CFCD0A124E400884204D28025ED00FC
:1021100018514019F8E70021995030BD00E0014006
:102120000405000010B5002804D19020922100027F
:10213000890203E0922080218002C902FFF7D8FFC4
:1021400010BD002802D092239B0201E090231B02C5
:102150001B6800201A0E532A01D11B02180A70476F
:1021600030B501248025064A064BED00D450545961
:10217000002CFCD001600021014AD15030BDC04686
:1021800000E001400405000010B5002802D09220B4
:10219000800201E090200002A6230902DB05090A63
:1021A0001943FFF7DDFF10BDF0B5012480250300C2
:1021B0000F4F08000F49ED007C507C59002CFCD0DB
:1021C0009C46002810DD5478167893782402344316
:1021D0001B0423431C00D37801381B0623436446A9
:1021E00008C40432A446ECE700237B50F0BDC0468F
:1021F00000E001400405000070B505004B680A00CE
:102200009C1C2100FFF7D0FFA000281870BD000023
:10221000154B1B68002B04D080219223C9029B021E
:1022200003E09221902389021B02002807D1191D87
:102230005B6802001B0E522B14D10A0012E0002230
:1022400081420FD903681B0E522B0BD14368023316
:102250009B00C318994205D91A68110E0022522911
:1022600000D11A0010007047F00600208022F0B55F
:10227000520085B00021624802F0F5FF8022002163
:102280005200604802F0EFFF5F4B1B681A00029398
:1022900053425A4110000392FFF744FF029B002B68
:1022A00001D15A4C00E05A4C0020FFF7B1FFFF2744
:1022B0000500002D00D194E02B681A121B143A403F
:1022C0003B4001921A000A3A092A43D84C4B019A22
:1022D000995C002900D07FE010224E4802F0C3FF35
:1022E0002E00336801991A123A40914217D11A14FC
:1022F0003A400B2A06D0132A0CD00A2A0FD1454B9C
:102300001E600CE03B40022B09DC424A9B00D318C4
:102310005E6004E0102200213E4802F0A4FF30007D
:10232000FFF776FF061EDCD13A4B196800290FD063
:102330002000FFF761FF0400374E3168002903D009
:102340002000FFF759FF0400344B0436B342F4D1A8
:102350002B4B3EE0143B092B3ED82A4B019A995C4B
:10236000002939D108222E4802F07DFF2E00336863
:102370001A143A40152A0BD01D2A11D0142A14D150
:10238000019A1B123B409A420FD1254B1E600CE074
:10239000019A1B123B409A4207D1214B5E6004E038
:1023A000082200211E4802F05EFF3000FFF730FFD8
:1023B000061EDCD11A4E3168002909D02000FFF733
:1023C0001BFF71680400002902D0FFF715FF04000D
:1023D0000C4B0121019A99542800FFF719FF0500C1
:1023E00067E70298FFF7ADFE411C0398FFF7CCFEAC
:1023F000054B039A1A600B4B1C6005B0F0BDC0463C
:10240000F0050020F0040020F0060020044802003F
:1024100004900000481F00204C1F0020581F00207F
:10242000581F0020F406002070B50020FFF789FE39
:1024300004000120FFF785FE844200DA04000A4B05
:102440001E687542754128001D60FFF76BFE002E67
:1024500001D0064B00E0064B064A2800611C1360C1
:10246000FFF792FE70BDC046F00600200490000009
:1024700004480200F4060020F8B50020FFF761FED2
:1024800007000120FFF75DFE3E00224D0643224C6F
:102490000CD180219020C9020002FFF729FE012102
:1024A0003000FFF771FE2E601C4B2FE0874208DDE5
:1024B000002392212B60194B89022360236800209E
:1024C00011E0012380212B60154BC9022360F5E741
:1024D0001A68551C18D0120E522A07D101205A68CA
:1024E000023292009B188B42F2D311E0002800D0F8
:1024F00023600C4C0C49200003F0DAFA200000F0B5
:10250000A7FEFFF791FF04E0002802D0236000E05F
:102510002160F8BDF0060020F406002004900000C1
:1025200004480200601F0020B16A0000F0B585B0C9
:10253000039203220333DC1714402A4EE3189C1045
:10254000336801900291002B02D08022D20201E078
:1025500092229202244FA51C3B68AD005B199A425F
:1025600017D2FFF783FE3368002B02D08022D202FD
:1025700001E0922292023B685B199A4209D21B4CFD
:102580001B49200003F094FA200000F061FE0020B7
:1025900026E0029B3E681B06190C6B461A7BA4239F
:1025A000DB051343019A0B431104FF22120411406F
:1025B00019433000FFF7D4FD3300301D08332100EC
:1025C00001933B60FFF7CCFD002C04D00A9A210058
:1025D0000198FFF7E9FD3000019B083D5D193D6062
:1025E00005B0F0BDF0060020F4060020601F0020BA
:1025F000DA6A000070B59AB0FFF73EFFFF221F4C69
:10260000D2000021200002F02EFE0020FFF700FE85
:10261000FF25002600281AD003681A142A400A2A27
:1026200008D11A122A40FF2A0ED0D200A1180B712D
:10263000A05009E0132A07D11B122B40FF2B03D017
:10264000DB00E2181671E650FFF7E2FDE2E7FF213A
:102650000200C900235808305D1EAB41D2188842E1
:10266000F8D1074901A803F0F7F901A800F062FAD0
:10267000044800F05FFA1AB070BDC046EC160020A6
:10268000016B0000196B0000044A05491368C85427
:1026900001339B059B0D13607047C046FC0A002068
:1026A000F8060020114A70B51368114C984211DAEF
:1026B000015D451CFA39012906D8AB4206DD211817
:1026C000497801391F2901D92800EFE70100251AAF
:1026D000461C02D10023136006E0665C6E54013193
:1026E0008B42FADC181A106070BDC046000B002047
:1026F000080B002010B500F099FD064B1A689042B7
:1027000001D200221A601B68C01A034B8342804129
:10271000404210BD040B0020204E000010B5094CB3
:10272000094A2368126893420BD0084AD05C00F033
:10273000B9FE002805D0236801339B059B0D23605B
:10274000EDE710BD080F0020FC0A0020F80600206D
:1027500010B50400064B074A1B6812689B1ADB433E
:102760009B059B0DA34202DAFFF7D8FFF2E710BDED
:10277000FC0A0020080F0020F7B506000191151E85
:102780002FD05768B800441C0630FFF7E1FFFB204C
:10279000FFF77AFF1C20FFF777FFF0B2FFF774FF17
:1027A000E0B22412FFF770FFE0B2FFF76DFF6B4657
:1027B0001879FFF769FF0026BE4212DAB300EB1862
:1027C0009C680136E0B2FFF75FFF2012C0B2FFF74E
:1027D0005BFF2014C0B2FFF757FF200EFFF754FF36
:1027E000EAE7F7BD70B5074D2C68042C08DC0C2314
:1027F0006343054E01349851F31859609A602C6078
:1028000070BDC0460C0F0020C41F0020F0B589B079
:1028100004900E0001284BDD284B086802938307C3
:1028200009D1042807D90F2302681340042B02D1D1
:10283000FFF74CFC0290214B70680393830709D18A
:10284000042807D90F2302681340042B02D1FFF795
:102850003DFC039000271A4B1A4D1B680593059BFE
:102860009F4225DA2B1F0299186803F017F90028F8
:102870001BD12B686C6806930190019B069A9342CA
:1028800013DA20680399079403F008F90834002844
:1028900007D131000498079B08315B6802389847DC
:1028A00009E0019B01330193E7E701370C35D6E7D7
:1028B0001B20FDF7A9FE09B0F0BDC046406B00002B
:1028C0000C0F0020C81F002010B501F021FA00F005
:1028D000A9FD00F015FE01F07FFA01F0A9FB10BD83
:1028E000C82210B5D2000021034802F0BCFC00222F
:1028F000024B1A6010BDC046AC10002098010020A9
:10290000064B074A1B6812689B1ADB439B059B0D0D
:102910000122834200DC002210007047FC0A0020E4
:10292000080F0020F8B505000C0016001F1E0ED180
:102930000320FFF7E5FF002827D0FA20FFF7A4FEC9
:10294000E8B2FFF7A1FEE0B2FFF79EFE1DE0501DCA
:10295000FFF7D6FF002818D0FB20FFF795FEE8B25E
:10296000FFF792FEE0B2FFF78FFEF0B2FFF78CFEAA
:102970003012C0B2FFF788FE3C00E31B9E4204DD2C
:102980002078FFF781FE0134F7E7F8BD70B5002429
:10299000A0250B4B1B689C420EDA2A006243094BB0
:1029A000D3181A78002A05D05978002311201A006C
:1029B000FFF7B8FF0134ECE7FFF792FF70BDC046A8
:1029C00098010020AC1000200123F3B50400FFB0F3
:1029D0000D0010001A420DD002AA1370431002A974
:1029E000537042121B0E40148A700B71C8700B009A
:1029F000052273E0032313401ED1042A1CD90F22A1
:102A000001680A40042A17D1023302AA1370FFF7A3
:102A10005DFB060003F054F8F823FF33984200DD15
:102A200018000023834205DA01335A1EB25C02A962
:102A3000CA54F7E7421C50E0042801D0002809D10D
:102A4000032302AA04381370434243415370130016
:102A5000022243E0002B45D1042843D90F2102680C
:102A60001140052912D1043302A90B70F823120971
:102A7000FF3392009A4200DD1A00002393422BDAC2
:102A80000133C118C97802AEF154F7E7062929D1FC
:102A900001390E00120956430196F826019FFF36B0
:102AA000B7421FDC02AE31700136934213DA0127C0
:102AB000013399004158394201D0394100E00A49B7
:102AC000012737700F127170B7700F14090EF7706D
:102AD00031710536E9E7019A013202AB2900200085
:102AE000FFF720FF7FB0F3BD19FCFFFF70B5A023F7
:102AF000050000240D4A1800604380184178A9425F
:102B000003D001340A2CF6D10FE0A022002102F0FC
:102B1000AAFB074A1368013BA34200D114600023BB
:102B200029001A001120FFF7FDFE70BDAC10002037
:102B30009801002010B5B2B002236A460400137059
:102B400002F0BEFFC72800DDC7200023834205DA5C
:102B5000694601335A1EA25CCA54F7E7421C6B4611
:102B6000FF211420FFF7DEFE32B010BDF7B5234B76
:102B700006001B68A020009300232149009A93427D
:102B80000ADA02005A438A185478B44202D1127801
:102B9000002A31D10133F1E70024A0231A00624357
:102BA00001920199164A55182F78002F06D001344A
:102BB0000A2CF3D11348FFF7BDFF1DE0A022390016
:102BC000280002F050FB02230D4A0199EB60535498
:102BD0000D4AF1008A58009B6E70AE70AA602F619A
:102BE0006F61A34202DC054B01341C6000233100FD
:102BF0001A001020FFF796FEF7BDC046980100208E
:102C0000AC100020D46B0000EC16002010B5FFF7CC
:102C1000BDFE0024064BE200D3181B79043B012BB8
:102C200002D8E0B2FFF7A2FF0134FF2CF2D110BDB1
:102C3000EC160020F7B50E0000247F250190194BFB
:102C4000E200D1180979062901D0032926D1985824
:102C500083682B401C2B21D1C3681A002A40042A08
:102C60001CD102692A40192A18D11B0A01339B0082
:102C70000C30C018FFF72AFA070002F021FF0023EA
:102C8000B0420BD19E4206DD019AF95CD25C9142C2
:102C900004D10133F6E7E0B2FFF768FF0134FF2CFF
:102CA000CDD1F7BDEC16002070B500F0BFFA184B7F
:102CB0001A68904201D200221A601A681549821AD5
:102CC0008A4223D91860002000F082FB444244412C
:102CD000604207240443002000F08EFB002810D03F
:102CE000082600250C4BEA00D3181B799C4201D022
:102CF000B34202D1E8B2FFF739FF0135FF2DF1D120
:102D000004E0631C02D001267642EAE770BDC046AB
:102D1000F80A00200F270000EC16002037B5002429
:102D20000500FFF733FE01A8019400F03FFB2000EF
:102D300000F068FE00F0FCFC00F072FB00F071FB9C
:102D400000F038FF00F09EFA0548FFF7F3FEA542B9
:102D500004D0FFF71FF90348FFF7ECFE37BDC0466C
:102D6000E96B0000016C0000002310B501001A009F
:102D70001120FFF7D7FD10BD07B56B4619706946E6
:102D80005A7013128B701314120ECB700A716B46AB
:102D9000010005221320FFF7C5FD07BD10B50A008D
:102DA00001001220FFF710FE10BD70B505000800ED
:102DB0000C003230FFF7CCFC2B00220000211B203E
:102DC000FFF7B0FD70BD10B50C000300110014201A
:102DD0002200FFF7A7FD10BD70B506000020FFF729
:102DE00017FA0024FF25002810D003681A142A407F
:102DF000152A05D11B122B40B34204D1040002E076
:102E00001D2A00D10024FFF703FAECE7200070BD73
:102E1000F0B580279DB0FFF781FCB94DB94C28680B
:102E2000FF00391A201800F023FB2B680600C31896
:102E30002B60002B00D1DBE1002E0DDD2868391A54
:102E4000201800F015FB2B6806001B182B6000F003
:102E5000EDF9AD4B1860EFE72378FA2B00D00CE1C9
:102E60002B68022B06DCFFF745FC002800D1BFE1F0
:102E70000120B8E16078A5780238182800D9FAE076
:102E800001F0BCFF0D1E22262932F93D676F7589BE
:102E9000DAEFF9F9F9F9F9F9F9F9F9F9F300FF2D90
:102EA00000D1E8E02800FFF721FE00229749EB005F
:102EB0005A50CB181A7129000092130013204DE0CC
:102EC0002800FFF753FED6E02800FFF70FFED2E000
:102ED000FFF79CFECFE0FFF759FD0020FFF71EFF34
:102EE0008B48FFF727FEC6E0182D00D9C3E0894BB9
:102EF000AA00D25829001520FFF766FDBBE0002488
:102F00002000FFF769FF071E03D10134192CF7D108
:102F1000B1E0083002F0D4FD06000530FFF718FCE0
:102F2000FB20FFF7B1FB1D20FFF7AEFBE0B2FFF780
:102F3000ABFBF0B2FFF7A8FB3012C0B2FFF7A4FB67
:102F40000025AE42E1DD7B19187AFFF79DFB0135C4
:102F5000F7E700211D200B000A000091FFF7E6FAB9
:102F600089E000222900009213002720F6E700F0F4
:102F700077F903AC684A64210090684B200002F0A6
:102F800039FD02232000237002F09AFD2300020085
:102F9000002116206DE000245C4AE300D558002D86
:102FA00046D06B689E00701DFFF7D2FB2B000025FA
:102FB0003200083321000120FFF7B4FC0020FFF7A6
:102FC00027F92E002F0000281DD0FF2103681A12B8
:102FD0000A40A24214D11A140A400B2A07D10B400E
:102FE0000DD0012B09D0022B00D1FFE008E0132AFD
:102FF00006D100252E002F0002E0060000E00700A9
:10300000FFF706F9DFE7002E04D03200012120008F
:10301000FFF7B2FB002D04D02A0002212000FFF7A9
:10302000ABFB002F04D03A0000212000FFF7A4FBE7
:103030000134FF2CB0D11EE0FFF7A8FC00250024CE
:10304000290000942300220013200135FFF76EFAB7
:10305000FF2DF4D1FF222100D2002C4802F003F909
:1030600009E00120FFF75AFE05E0002329001A00BD
:103070001A20FFF757FC0320B5E0FB2B00D0F7E642
:103080002A68042A00DCEEE62679E078244B360232
:1030900006439E4200DDEBE6331D9A4200DCE2E689
:1030A000E35CFE2B00D0E3E66078A578731E1C2855
:1030B00068D007D8082835D01B285ED0012800D05A
:1030C00090E007E01E2800D17EE066D31F2800D1E3
:1030D00080E087E0FF2D00D184E02800FFF706FDA7
:1030E00067790634B31E290000943A000A20FFF7DE
:1030F0001DFA064BED00E8505D192F7172E0C046D5
:10310000000B0020080B0020040B0020EC16002010
:10311000116C0000E41E0020286C0000236C0000ED
:10312000F6030000182D5DD86079022813D003281B
:103130001BD0012856D1A71D7A78A479BB7812023A
:1031400022431B0413431A00FB78AD001B061343F4
:103150005B0003430EE0002B44DDB11EA01DFEF713
:1031600099FF244BAD00E8503CE0A379AD005A1E16
:1031700093419B001F4AAB5034E0601D1900FFF7DC
:1031800059FD2FE0FF2D2DD06279022A2AD806346E
:10319000B31E009429000B2022E0632B00DD632383
:1031A000002203A8934204DDA11849798154013219
:1031B000F7E7D9430022C917194041180A700133B3
:1031C0000090290015200BE005340094002229000E
:1031D0001E2005E0042B05D10022290005340094AF
:1031E000FFF7A4F9701DFFF75DFA01E0050007E79E
:1031F0001DB0F0BDE41E0020002070470020704785
:10320000002070470020704701220020054B06492E
:103210001A61585003300431585080180831585002
:103220001A60704700800040040500000122034B33
:103230001A64A822D20098587047C0460080004007
:1032400010B5FFF7F3FFFA21890001F0E1FD10BD91
:1032500010B50100014801F085FB10BD38100020B9
:1032600000487047386C000070B5054E0400335CB0
:103270000D008B4202D001F09DFA355570BDC0465D
:10328000100F002070B50024064D635D012B05D1A1
:103290000021200001F08EFA0023635501341D2C1B
:1032A000F2D170BD100F00200D2070473B207047F9
:1032B000036870B55B100120052B12D8094A9B00EA
:1032C0009C58094D2B5D002B05D00021200001F0FA
:1032D00071FA00232B55200001F016F9012340005C
:1032E000184370BD686C0000100F002070B50368B3
:1032F00045685C106D1004D40B4B9D4202DD1D002F
:1033000000E000251C2C0DD8084E335D012B05D0A4
:103310000121200001F04EFA01233355290020003D
:1033200001F080F970BDC046FF030000100F0020BF
:1033300070B5046864101C2C0FD8094D2B5D002B50
:1033400005D00021200001F035FA00232B55200084
:1033500001F064FA0423012800D00023180070BD96
:10336000100F002070B504000D001C280ED8084E68
:10337000335C012B04D0012101F01CFA01233355E9
:10338000290020004D1EA94101F032FA70BDC0464F
:10339000100F0020436810B5191F4A424A410068C7
:1033A00011004010FFF7DEFF10BD000037B5694681
:1033B0000200064B684630CB30C11368042B02D1A3
:1033C00000F030FB01E000F055FB37BD306C000031
:1033D00010B5084C6379002B05D00021052001F0C1
:1033E000E9F900236371052001F018FA43425841BE
:1033F000800010BD100F002010B5084CE37A002BA0
:1034000005D000210B2001F0D5F90023E3720B2039
:1034100001F004FA43425841800010BD100F002013
:103420007047704710B5034A04210348FFF7DAF9E3
:1034300010BDC04604000020426C0000E12110B520
:103440004902094801F0D5FAFFF7DEFE0A2001F033
:1034500055F80023FF21054A995401331D2BFBD158
:1034600000F0A8FB10BDC04638100020100F00204F
:10347000F8B50B4E070030000D0001F0F9FA041EFC
:10348000AC4200DD2C003D00EB1B9C4205DD300012
:1034900001F0F8FA28700135F6E72000F8BDC046C3
:1034A0003810002010B50100014801F0A9FA10BD44
:1034B000381000200020704710B51E20FDF7A4F83A
:1034C00010BD10B51E20FDF79FF810BD10B51E20D1
:1034D000FDF79AF8002010BD10B51E20FDF794F8F6
:1034E00010BD10B51E20FDF78FF810BD10B51E20C1
:1034F000FDF78AF810BD10B51E20FDF785F810BD48
:1035000010B5034A08210348FFF76CF910BDC04607
:1035100024000020806C00000123034A1360034A4A
:103520001068984018437047380F0020400F002063
:10353000202800D90020084B8000C2580123934066
:10354000064A07491360074A1160074A0749116094
:10355000074A13607047C0461C710000340F0020FA
:1035600008050050500F0020480F00200C050050A7
:1035700018050050F0B5EFF310810123194083F3D3
:103580001088134E134AB4461268013A9340124A07
:103590001468124A1568124A002B15D016680342A7
:1035A0000BD02660C046C046C046C046C046C04696
:1035B000C046C04616682E6004E067463E60166846
:1035C000084F3E605B08E7E781F31088F0BDC04616
:1035D000080500506C000020500F0020480F00200C
:1035E000340F00200C05005030B585B001AD0C2221
:1035F0000649280001F02EFE0024285D0121013437
:10360000FFF732FE0C2CF8D105B030BDF66C00008F
:10361000F0B53B4C85B0210003220C31684601F027
:1036200019FE210009220F3101A801F013FEFFF756
:1036300007FE344B344CC0182368984201D2002353
:1036400023602568002D3ED12E006B4604339F5D1C
:1036500001213800FFF708FE01360121380001F092
:10366000C7F8092EF1D100266B469F5D0121380075
:10367000FFF7FAFD01360021380001F0B9F8032EFA
:10368000F2D1C82080000138C046C046C046C046BE
:10369000C046C046C046C046C046C046C046C046FA
:1036A000F1D100210420FFF7DFFD00266B46002149
:1036B000985D0136FFF7D8FD032EF7D1FFF7C0FD67
:1036C0001330206019E0FFF7BBFD23680025984206
:1036D00013D3042000F018FF0C4B0D4EC01801D47A
:1036E000306000E035603068032101F01BFC0023EE
:1036F0000125084A306023601360280005B0F0BD42
:10370000F66C000010270000300F0020C8FEFFFFFD
:10371000400F0020380F002010B50124044001D0D4
:10372000441002E00D20FCF76FFF200010BD0000E8
:103730007FB5A44E3368002B0BD1A34A1268002A30
:1037400007D1A24B1B68002B00D139E1FFF760FFC6
:1037500036E19F4D2A68002A2AD19C4A1268002A25
:1037600007D0FFF755FF002800D129E1FFF73CFF04
:1037700005E0954A1268002A01D1002BF6D1924B40
:1037800019681A00002911D03468002C0ED101AD3F
:103790000C22904928001C6001F05CFD285D00218E
:1037A0000134FFF761FD0C2CF8D109E13368136097
:1037B00000211A2001F01CF800211B2001F018F84C
:1037C00000211C2001F014F82E68012E56D0022E84
:1037D00000D19CE0002E00D0ECE0013631007A4CA4
:1037E00003202368994301F003F804202168014075
:1037F0000B005942594100F0FBFF102123680A20B9
:103800000B405942594100F0F3FF80212368090120
:103810000B4059425941062000F0EAFF80212368FD
:1038200009020B4059425941072000F0E1FF802175
:10383000236849020B4059425941092000F0D8FF42
:103840008021236889020B4059425941192000F018
:10385000CFFF80212368C9020B40594259411820EB
:1038600000F0C6FF802321681B030B4059425941D9
:10387000172000F0BDFF31001A2099E00221524CC0
:10388000172023680B405942594100F0B1FF08212D
:10389000236818200B405942594100F0A9FF8021AC
:1038A0002368C9000B4059425941042000F0A0FF91
:1038B0008021236849010B40594259410A2000F0F8
:1038C00097FF80212368C9010B40594259410320C9
:1038D00000F08EFF8021236889030B405942594133
:1038E000092000F085FF802321681B040B4059420A
:1038F0005941192000F07CFF3100062000F078FFCC
:103900003100072000F074FF31001B2050E020211F
:103910002D4C172023680B405942594100F068FF95
:103920004021236818200B405942594100F060FFA4
:103930008021236819200B405942594100F058FF5B
:103940008021236849000B4059425941092000F069
:103950004FFF8021236889000B40594259410720BD
:1039600000F046FF8021236889010B4059425941EC
:10397000062000F03DFF8021236849030B40594297
:1039800059410A2000F034FF80212368C9030B400D
:1039900059425941032000F02BFF802321685B042A
:1039A0000B4059425941042000F022FF01211C2004
:1039B00000F01EFF2B680321581C01F099FB2960C1
:1039C0007FBDC046440F00203C0F0020380F002070
:1039D0004C0F0020F66C0000006810B5C30703D53B
:1039E000FFF79AFE054B1860054B1B68002B03D0B0
:1039F000024B186800F01AFB10BDC046440F0020AF
:103A0000580F00200022054B10B51A60044B1B68AC
:103A1000934201D000F008FB10BDC046440F0020C7
:103A2000580F002070B505000068FFF775FE040010
:103A30006868FFF771FE631E0100042B14D8451E51
:103A4000042D11D805226A43D318012215009D4088
:103A50002B00064805682B430360054B1B68002BB1
:103A600002D0200000F0E1FA70BDC046440F0020F3
:103A7000580F002070B505000068FFF74DFE0400E8
:103A80006868FFF749FE631E0100042B14D8451E29
:103A9000042D11D805226A43D31801229A4013003D
:103AA000064802689A43064B02601B68002B03D04D
:103AB0000022200000F0B9FA70BDC046440F00207B
:103AC000580F00202C4BF7B51B680400002B03D1C6
:103AD00001204042FFF72CFD01262468344219D012
:103AE000FF226310180212041040FF22611212021A
:103AF0000A40DBB210431843204B1B68202B06D131
:103B0000B4401F4BA40EA400E35800021843FFF773
:103B100031FD30E0032525402DD1042C2BD90F2376
:103B200022681340062B26D1FF27130901933F0477
:103B3000019B9D421FDAAB00E3185A68324218D04D
:103B4000531018023840FF218446090250120840E1
:103B50006146DBB208431843084B1B68202B06D193
:103B60005200920E064B9200D35800021843FFF702
:103B700001FD0135DCE7F7BD500F00206C0000208F
:103B8000246D00000B6810B50200D80701D558104D
:103B900001E0012040421823012A03DD4A68042A7B
:103BA00000D10833024A1360FFF7C2FC10BDC046C3
:103BB0006C000020012010B54042FFF7B9FC10BD99
:103BC0000068F8B5C30702D5FFF7A6FD0BE0830731
:103BD00026D1042824D90F2203681A40042A1FD1B1
:103BE0001B091DD000790300203B5E2B18D805224D
:103BF000002053430B4E9D18043AAB420CD00521D4
:103C000010249F5D3C4200D080180139520064109E
:103C10000029F7D10133F0E701234000184300E009
:103C20000120F8BD246E0000F0B5050085B00868DD
:103C30000C00FFF771FD0390022D08DD6068FFF7AF
:103C40006BFD0700A068FFF767FD040001E0012499
:103C5000270005236343053B0293012326000193BC
:103C6000231D9E4234DC3D003B1D9D422BDC731E18
:103C7000042B23D86B1E042B20D8029B039A591EB9
:103C8000019B49191A40204B0AD001228A40196829
:103C90000A431A601D4B01221B68002B0ED009E05D
:103CA000012088400100186888431860174B1B6882
:103CB000002B03D03100280000F0B7F9019B01353B
:103CC0005B000193D0E7029B013605330293C7E7FF
:103CD0003D1D042D15D8012C13D126003300AB4017
:103CE000094A11689943094B11601B68002B04D0E5
:103CF000781D0022210000F098F901340535062CCA
:103D0000ECD105B0F0BDC046440F0020580F002094
:103D100010B5034A01210348FEF764FD10BDC046FB
:103D2000640000200E6D00000122094B1A60094A50
:103D30001368002BFCD00322074B1B68D8171040D8
:103D4000C018012380100638400018437047C04651
:103D500000C0004000C1004008C50040012070477D
:103D600010B501210D20FFF77FFA01210E20FFF78A
:103D70007BFA00210F20FFF777FA044C200000F0B7
:103D8000C9F91021200000F0E1F910BD680F0020F2
:103D900010B504680D20E30703D56410FF2C03D988
:103DA0001720FCF731FC06E0FFF7DAFFE1B202482A
:103DB00000F0EEF9002010BD680F002010B5FFF7ED
:103DC000CFFF0021034800F0E3F90123400018432E
:103DD00010BDC046680F002010B5034A05210348F6
:103DE000FEF700FD10BDC04674000020FF6F00000C
:103DF000F7B50F4F06003B680D0001920D4C002BEC
:103E000004D1200000F04AFA01233B60F1B2200007
:103E100000F0D2FAE9B2200000F001FA6B4620006F
:103E2000197900F0FCF9200000F030FBF7BDC04626
:103E3000540F00207C0F002010B50124036823429A
:103E400005D04168214202D08268224201D10D2072
:103E500004E058104910802803D91520FCF7D4FB42
:103E60000BE0FF2901D91620F8E75210FF2A01D9EB
:103E70001720F3E7FFF7BCFF002010BDF8B5154F82
:103E800005003B680E00144C002B04D1200000F00C
:103E900005FA01233B60EDB22900200000F08CFA06
:103EA000F1B2200000F0BBF90021200000F090FAF0
:103EB000002801D040420CE001222900200000F03F
:103EC00076FA200000F0A1F90028FAD0200000F0D6
:103ED000A1F9F8BD540F00207C0F002010B501247B
:103EE0000368234202D04168214201D10D2004E041
:103EF00058104910802803D91520FCF785FB07E0EE
:103F0000FF2901D91620F8E7FFF7B8FF400020434A
:103F100010BD0000002370B5344D0400EB56013392
:103F20002BD10D211D20FFF7A9FF5A2804D1012212
:103F30002A212A703D380AE00F211920FFF79EFF41
:103F4000332807D102235F2220212B701A38FFF774
:103F50004FFF12E00D211E20FFF790FFC7280AD166
:103F6000032300222A21A9382B70FFF741FF1B22CF
:103F70002A211E20EBE700232B700023EB56022B97
:103F800006D0032B13D0012B26D121001D2010E0D9
:103F9000012C04D129211920FFF770FF0DE0032C1B
:103FA00015D12B211920FFF769FF043C05E0210002
:103FB0001E200124FFF762FF64427F2801DD0138E3
:103FC000FF3803007F330ADA7F20404207E0052CE8
:103FD00002D12D211920ECE7012400206442642342
:103FE0007F21584300F09EFF604370BD70000020A9
:103FF00010B50120FFF78EFF01234000184310BDCC
:1040000010B50320FFF786FF01234000184310BDC1
:1040100010B50520FFF77EFF01234000184310BDB7
:1040200000207047002070477047704770470000BD
:1040300010B5034A02210348FEF7D4FB10BDC04669
:104040009C0000202F70000010B5FFF7F7F906481C
:10405000FDF7C2FFFEF738FC0448FEF76BFDFEF7E4
:10406000C9FAFEF7D3FD10BDD6060000E96B0000CB
:1040700010B5FDF743FF10BD70B5002504AC2478E2
:104080000573A94205D10A4B0A4A23210A4801F0C7
:1040900061F801600949920052589B0002715B5817
:1040A0008371A3005B58856043710223C37170BDA7
:1040B000877000004A700000957000001C710000BD
:1040C000037B002B04D143738373036101330373B8
:1040D000704700001FB50191A02100240068C900AD
:1040E000D2B24450012A07D0A24203D0032A05D1FC
:1040F000042202E0022200E006221343034A835016
:10410000034B019AC250012343501FBD54050000C8
:104110002405000010B50400FFF7D2FFA122236898
:10412000A179D20099506179064A200099502179ED
:1041300004329950044B19685A689B68FFF7CAFF0C
:1041400010BDC0460C0500005C0F00204BB2002BD8
:104150000CDB80233F290CD81F290CD80F290CD841
:1041600007290CD803290CD81B060BE080239B04DD
:1041700008E0DB0406E01B0504E05B0502E09B05AC
:1041800000E0DB050168014A8B5070472405000000
:104190000368074A99501A00FC32D1680029FCD004
:1041A000A321C90058580023C0B2D3607047C0464D
:1041B0001C05000007B58022074BD2051A600022BB
:1041C0009A6002321A710F230C3200930349023BAA
:1041D0000348FFF751FF07BD5C0F0020003000408F
:1041E000680F0020F8B505000E0017000024BC423F
:1041F00008D02B68315D1B6828009847002801D043
:104200000134F4E72000F8BD704710B51C3000F011
:10421000D5FB10BD10B51C3000F0C2FB10BD70B551
:10422000437E0D00002B05D06430040000F0D5FB68
:10423000002801D0002004E02000290000F0A1FBAC
:10424000012070BD10B51C3000F0BEFB10BD000099
:10425000F7B50193FA23002504009B0083600D4B02
:104260004560083303601C300F00160000F07EFB31
:104270002000643000F07AFB074AB600B35827618B
:104280006375019B20009B009B586576A576A375FE
:10429000FEBDC046FC7000001C7100000123A0227E
:1042A000C375837D0C49C133FF33D2059B00995000
:1042B000437DC133FF339B009950CC210369074AEA
:1042C000490499500521243A9950817D083299502A
:1042D000417D034A995070470C06000024050000F8
:1042E0000C050000F7B5050000200C000193824288
:1042F0005CD0161E402E00D940262F001C373800F7
:1043000000F04AFBB1222B69D20080219C5001228F
:1043100089005A50A97E002901D11A621A6000242E
:10432000731E2A69A34206D1019B002B03D0802370
:1043300002219B00D150012313621300FC33D96882
:10434000002902D1996A0029F9D0996A00290AD175
:10435000D960A323DB00D1583800C9B2013400F082
:1043600010FBA642DCD8019A2B69002A04D11A005E
:10437000FC32916A00290AD001210022AA765961F3
:104380001900FC3188680028FCD08A6007E0012110
:10439000A976D961D16C0029FCD00021D164FC330D
:1043A0009A6A002A01D000229A62E0B2FEBD10B5DE
:1043B0000123FFF797FF10BD0300AC3310B50400D5
:1043C0001970643000F0E8FA0123637610BD000034
:1043D000F8B500220D0001004276AC3103690400FB
:1043E0000878B121C9005850802189005A50013203
:1043F0001A629A6026006436300000F0DFFA002866
:104400000ED03000276900F0CBFA1E4BF85023691C
:10441000FC331A6A002A0CD19A6A002AF9D008E003
:104420002369002D0AD11A00FC32916A002905D1B6
:104430000EE09A6A002AF3D11A62DBE701225A6180
:104440001A00FC3291680029FCD00021916006E03E
:104450000121D961D16C0029FCD00021D1641A005E
:104460000020FC32916A81420BD0074990625A5871
:1044700002305A50824204D0043A5342534102302F
:10448000C01AF8BD1C050000C404000010B50121CD
:10449000FFF79EFF10BD000010B513231422024940
:1044A0000248FFF7D5FE10BD004000407C0F002001
:1044B00003210A4802680A430260094802680A4365
:1044C00002600849084A094B9B1A03DD043BC8589F
:1044D000D050FBDC00F0B4F9FBF74CFE24050040A3
:1044E00054050040B4730000000000207801002053
:1044F000FEE7FEE7FEE7FEE7FEE7FEE7014B18609A
:104500007047C046B4000020F7B50023202877D8B4
:104510003C4B8000C258042A14D006D8022A0DD081
:104520000ED80423012A14D069E0062A0ED00BD33A
:104530001A2A0DD002231B2A0BD060E0082308E0C2
:10454000102306E0202304E0402302E0802300E063
:1045500001232D4A1268082A04D9092A05D00A2104
:10456000022404E00821002401E011000124A02518
:1045700001261C272548ED004651254D254E2D6866
:104580001B02AD003D400195234D2D6800958559D6
:10459000AC466746214D3D401D4385518359C0259A
:1045A0009C46009BAD021D40FF2367461B023B401B
:1045B0002B43019D1D43009B5F0160231F402B0087
:1045C0003B431C4301238451154C036063680F482F
:1045D000002BFBD00024124B01255C60A123DB00E3
:1045E000C3584560A025ED0044511BB2914207D04D
:1045F00002D98A1AD34003E0521A934000E0002304
:104600001800FEBD1C710000B800002000700040C2
:10461000B000002004050000AC000020FF00FFFFF8
:10462000FC700040F0B520286CD8374B8000C25891
:10463000364B1E68002E2ED1C2243548A4000759DF
:10464000344B03253B40C0273F023B4303518023AB
:10465000893C9B00FF3C03512F4F03602F4B803C54
:10466000D859FF3CA043D8510437D859A843204318
:10467000D8510837D8590C35A843083D2843D8519C
:10468000A820C0001E508026C120760280001E5047
:104690001C601E4B1C6000231426214834005C4320
:1046A000255804006F1C0FD1142058432250A0201D
:1046B0000325C132FF329200C0051550194A080087
:1046C0001268082A03D10BE0AA4218D1ECE7082AA5
:1046D00002D9083AD14002E00820821A914008002D
:1046E00014225343E3189A680C495132FF32920066
:1046F00058605050DA68C1239B00CA5002E0013371
:10470000032BCBD1F0BDC0461C710000341000203B
:1047100000E100E0FF00FFFF040500000090004002
:10472000BC000020B40000201E4BF0B5596C1800EE
:104730001D4A002914D0A025A12600230124ED053F
:10474000F600D1584F1C06D0D7187F68002F02D032
:1047500027008F40AF5114333C2BF2D10023436428
:10476000131DA02540329446002001240F4EED0574
:10477000DA680F49920057180A495218526C002AF9
:104780000CD01A1F1268511C05D01968FF2902D0DD
:1047900021009140A9513A00FC32506414339C45E9
:1047A000E6D1F0BDFC900040BC0000200C050000EC
:1047B0000090004000B5202816D80C4A83009B5872
:1047C000032911D8A0220800C133FF33D2059B0072
:1047D00000F014FB02080406002104E00C2102E0B2
:1047E000042100E00321D15000BDC0461C7100002F
:1047F00020280DD8074B8000C058A0220123D205E5
:104800008340002901D1044901E0A121C90053508E
:104810007047C0461C7100000C050000030000201A
:10482000202B0AD8A222A021D200C9058858034A09
:104830009B009B58D8400123184070471C71000012
:104840002D4B10B51A78012A19D12C4A126812077B
:1048500015D12B4AE0241168F022080010402142B3
:104860000BD128490968114209D12749274A11600B
:104870008021274A0902116001E03028F1D01A781E
:10488000012A0DD11D490968090709D1F0201C49E9
:1048900009680140402903D11A490968014223D01F
:1048A0001B68DBB2012B25D1144B1B681B0721D1E0
:1048B000134B1A68F0231A40A02A04D1114A126837
:1048C0001A4203D016E0D02A14D1F7E7114B1A6828
:1048D000012A03D1C022104B1A600BE00F4A1A6064
:1048E0001A68012AFCD1F5E7C1218020C900C00562
:1048F0004250D5E710BDC046E00F00F0E40F00F0D5
:10490000E80F00F0EC0F00F0DFFF07C004050040E7
:10491000186C004000EC064014EC06407593000053
:10492000F7B506000D000C008B180193019B671B67
:104930009C4207D0336821781B68300098470134C7
:104940000028F3D13800FEBD70B505000C00081E2C
:1049500007D001F0B5F82B6802005B682100280041
:10496000984770BD10B5FFF7EFFF10BD10B540229E
:104970000021040000F077FC00232000236463641E
:1049800010BD3F23026C10B5541C2340446C9C4264
:1049900001D08154036410BD002303644364704755
:1049A000436C026C934206D03F21C25C01330B4042
:1049B0004364100001E0012040427047036C406CEA
:1049C000181A00D540307047436C026C934201D0F6
:1049D000C05C01E0012040427047036C406C5A1CEF
:1049E0003F231340181A42424241D0B2704701207F
:1049F000704710B503681322DB69984710BD7047F4
:104A00000369054A9950FC331A6A002AFCD0002237
:104A100001201A627047C0461C050000030010B553
:104A20005C331A781F2313400122110099400D4B6B
:104A30000424D967C221036989005C505A60DA6096
:104A4000A0220021D20099500122074952425A5017
:104A5000064914305A500C395A5008315A50FFF751
:104A60009BFF10BD04E100E00C05000014050000F0
:104A700010B51430FFF7A2FF10BD10B51430FFF7CA
:104A8000A3FF10BD10B51430FFF78AFF10BD000062
:104A9000030070B55E331C780269604BD45003008C
:104AA0005D331C785E4BD450030061331C785D4B42
:104AB000012C0CD105005F352E78A225ED00565152
:104AC000050060352E78A125ED00565100E0002448
:104AD000D4509623DB00994238D996231B01994282
:104AE00037D996235B01994236D996239B01994287
:104AF00034D9E1239B01994232D99623DB019942B3
:104B000031D9E123DB0199422FD996231B02994227
:104B10002DD9E1231B0299422BD996235B0299429E
:104B200029D9E1235B02994227D9E1239B029942CB
:104B300025D93D4B994224D9E123DB02994223D95F
:104B4000E1231B03994221D8384B21E09E23DB024D
:104B50001EE09D231B031BE0354B19E0354B17E08E
:104B6000EC239B0314E0344B12E0344B10E0344B45
:104B70000EE0344B0CE0344B0AE0344B08E0344B8D
:104B800006E08023DB0403E0324B01E080235B0579
:104B90003149002453500423243953501100FC316F
:104BA000CC600C62C1210134890014605C309460D7
:104BB000535003781F202200D9B20840824080342D
:104BC0002648FF345BB20251002B13DA0F230B404F
:104BD000083B234C9B089B001B1903242140A14048
:104BE000FC348C40DD69A543C0248C40210029435E
:104BF000D96111E0194C9B089B001B19032421402B
:104C0000A140C025FC348C40AD005E59A643C024B1
:104C10008C40210031435951026070BD0C050000E9
:104C2000140500006C05000090D0030000D0BE0EFB
:104C300000B013000050270000A04E0000F07500E7
:104C400000509D0000F0EB0000903A0100E0D70119
:104C500000B0AF0300705F072405000000E100E032
:104C600000ED00E0F7B5009308AB1B780025019339
:104C7000FA2304009B0083600E4B456008330360F9
:104C800014300F001600FFF771FE23005C3327611C
:104C90001E70009B084A9B00995823005D331970D1
:104CA000019B20009B009A5823005E33DD701A7030
:104CB000FEBDC046A07100001C710000036910B564
:104CC0001A00FC32D2680400002A0AD0A322D200C3
:104CD00099581430C9B2FFF754FE00222369FC33FF
:104CE000DA6010BD10B50248FFF7E8FF10BDC046FE
:104CF00038100020162307B5022200930249013B19
:104D00000248FFF7AFFF07BD002000403810002029
:104D10007047000010B500F047F8FFF7F9FF0120D9
:104D200000F024F8FFF790F9FFF7A2F9024B002BEF
:104D3000FAD000E000BFF7E700000000084A094988
:104D4000094B10B51B688858FA22190A1B0618432C
:104D50009200002300F0D2F94904C00B084310BDB3
:104D600004050000001001409C10002070B5041ED6
:104D700009D0FFF7E3FF050000F014F8FFF7DEFFAE
:104D8000401B8442F8D870BD0022044B9A60044A4C
:104D900013680133DBB213607047C046FC1001405A
:104DA0009C10002070470000C421114A890050580F
:104DB000104B0340C020000203435350802391391D
:104DC0009B02FF39535013608023A3220021DB058F
:104DD000D20099500122A1209A60074BC0001950BF
:104DE000C120023180001950403019501A607047BC
:104DF00000E100E0FF00FFFF0010014002B4714637
:104E000049084900095C49008E4402BC7047C0460D
:104E1000002243088B4274D303098B425FD3030AF9
:104E20008B4244D3030B8B4228D3030C8B420DD30C
:104E3000FF22090212BA030C8B4202D3121209029A
:104E400065D0030B8B4219D300E0090AC30B8B42D8
:104E500001D3CB03C01A5241830B8B4201D38B0386
:104E6000C01A5241430B8B4201D34B03C01A52412B
:104E7000030B8B4201D30B03C01A5241C30A8B426E
:104E800001D3CB02C01A5241830A8B4201D38B0259
:104E9000C01A5241430A8B4201D34B02C01A5241FD
:104EA000030A8B4201D30B02C01A5241CDD2C3096F
:104EB0008B4201D3CB01C01A524183098B4201D3EB
:104EC0008B01C01A524143098B4201D34B01C01AD6
:104ED000524103098B4201D30B01C01A5241C3084E
:104EE0008B4201D3CB00C01A524183088B4201D3BD
:104EF0008B00C01A524143088B4201D34B00C01AA9
:104F00005241411A00D20146524110467047FFE714
:104F100001B5002000F0F0F802BDC0460029F7D02E
:104F200076E7704703460B437FD4002243088B4249
:104F300074D303098B425FD3030A8B4244D3030B20
:104F40008B4228D3030C8B420DD3FF22090212BAE5
:104F5000030C8B4202D31212090265D0030B8B4261
:104F600019D300E0090AC30B8B4201D3CB03C01A4B
:104F70005241830B8B4201D38B03C01A5241430B26
:104F80008B4201D34B03C01A5241030B8B4201D316
:104F90000B03C01A5241C30A8B4201D3CB02C01A81
:104FA0005241830A8B4201D38B02C01A5241430AF9
:104FB0008B4201D34B02C01A5241030A8B4201D3E8
:104FC0000B02C01A5241CDD2C3098B4201D3CB018F
:104FD000C01A524183098B4201D38B01C01A52413E
:104FE00043098B4201D34B01C01A524103098B4242
:104FF00001D30B01C01A5241C3088B4201D3CB002D
:10500000C01A524183088B4201D38B00C01A52410F
:1050100043088B4201D34B00C01A5241411A00D2BF
:1050200001465241104670475DE0CA0F00D0494228
:10503000031000D34042534000229C4603098B4298
:105040002DD3030A8B4212D3FC22890112BA030A20
:105050008B420CD3890192118B4208D389019211A2
:105060008B4204D389013AD0921100E08909C30927
:105070008B4201D3CB01C01A524183098B4201D329
:105080008B01C01A524143098B4201D34B01C01A14
:10509000524103098B4201D30B01C01A5241C3088C
:1050A0008B4201D3CB00C01A524183088B4201D3FB
:1050B0008B00C01A5241D9D243088B4201D34B0016
:1050C000C01A5241411A00D20146634652415B1058
:1050D000104601D34042002B00D549427047634639
:1050E0005B1000D3404201B5002000F005F802BD7E
:1050F0000029F8D016E770477047C046F0B54F4614
:105100004646C0B41604360C9946330005042C0CF0
:10511000070C150C63437E436F4365431C0CAD19AC
:1051200064199C46A64203D980235B0298464744F3
:105130006346250CEF191D044B464A4343432D0C8F
:10514000240464199918C91920000CBC904699468A
:10515000F0BDC0467FB51D000A4B06001B68D8682D
:10516000002A02D1084C230001E01300074C0293EF
:10517000009133002A000649019400F021F800F064
:1051800023FEC04658010020406B0000D071000093
:10519000DD710000084B10B50400002B02D0002187
:1051A00000E000BF054B1868836A002B00D09847C9
:1051B000200001F0F3FAC046000000001072000069
:1051C0000EB403B5010003AB044804CB006801939F
:1051D00000F016F902B008BC03B0184758010020CF
:1051E0000E4B70B500251E000D4CE41AA410A5420C
:1051F00004D0AB00F35898470135F8E701F0D0FA36
:10520000084B00251E00084CE41AA410A54204D047
:10521000AB00F35898470135F8E770BD60010020F6
:1052200060010020600100207001002010B5034BD8
:105230000100186800F066F810BDC0465801002053
:1052400010B5034B0100186800F016F810BDC046F9
:1052500058010020002310B59A4203D0CC5CC454FE
:105260000133F9E710BD03008218934202D0197090
:105270000133FAE77047000030B500293ED0043909
:105280000B68002B00DAC9181D4A13681400002BA4
:1052900002D14B60116031E08B420DD90A68881849
:1052A000834203D118685B6882180A604B602160F2
:1052B00024E08A4203D813005A68002AF9D11D68F5
:1052C0005C198C420BD10968691858181960824220
:1052D00014D110685268411819605A600EE08C426F
:1052E00002D90C23036009E008680C18A24203D11C
:1052F00014685268201808604A60596030BDC04682
:10530000A4100020032370B5CD1C9D430835060072
:105310000C2D01D20C2505E0002D03DA0C23002012
:10532000336040E0A942F9D81F4B1C681A002100E5
:10533000002913D00B685B1B0DD40B2B02D90B601B
:10534000CC181EE08C4202D1636813601AE04B68EF
:1053500063600C0016E00C004968E9E7134C236811
:10536000002B03D1300000F033FB20602900300017
:1053700000F02EFB431CD1D00323C41C9C43A0424D
:105380000AD12560200007220B30231D9043C31A49
:1053900009D05A42E25006E0211A300000F018FB12
:1053A000431CEED1BAE770BDA4100020A01000206D
:1053B000936810B5013B9360002B05DA9469A34212
:1053C00008DBCBB20A2B05D01368581C106019708B
:1053D000C8B201E000F02CFC10BDF8B506000F00CB
:1053E0001400D518AC4208D021783A003000FFF7FD
:1053F000DFFF0134431CF5D100E00020F8BD0000C0
:10540000F0B59FB006000F0002920593002804D06B
:105410008369002B01D100F0D3FD7F4B9F4201D166
:10542000776808E07D4B9F4201D1B76803E07C4B71
:105430009F4200D1F768BB891B070AD53B69002B47
:1054400007D0002306AD6B6120336B761033AB764B
:105450003DE03900300000F043FC0028F1D001208D
:105460004042D6E0059A111D12680591002A00DA23
:105470007FE00992013423782E2B00D18DE0217832
:105480000322684800F082FE002807D0654B2A6896
:10549000C01A4023834013432B6001342178631CDE
:1054A000062261480293297600F070FE002800D1A0
:1054B0009DE05E4B002B00D090E00722059B073358
:1054C0009343083305936B69039A9B186B61029CA5
:1054D0002378002B04D1029BE31A049312D003E03B
:1054E000252BF8D00134F3E7049B029A39003000F1
:1054F000FFF773FF431C00D186E06A69049B944662
:1055000063446B612378002B7ED00122002352423A
:105510006A6002A95432521801342B60EB60AB6010
:105520001370AB6521780522414800F02FFE00285A
:1055300008D03F4B2A68C01A0123834013432B60D5
:105540000134EFE72B68DA0604D55322202102A8A4
:10555000121811701A0704D553222B2102A8121811
:10556000117022782A2A00D17CE7099B00200A21A9
:1055700005E05242EA60022213432B607AE7227868
:10558000303A092A04D84B4301349B180120F6E72E
:10559000002800D16FE709936DE763782A2B0AD1C1
:1055A000059B02341A1D1B680592002B01DA0123AA
:1055B0005B42079363E700230A201A0001346B6003
:1055C00021783039092904D8424301345218012383
:1055D000F6E7002B00D152E7079250E705AB0093A6
:1055E0003A00144B2900300000E000BF07E005AB93
:1055F00000933A000F4B2900300000F08BF8039025
:10560000039B013300D05EE7BB895B0600D526E72C
:105610000B981FB0F0BDC0464873000068730000CF
:10562000887300001A7200001E7200000000000063
:1056300014720000DB530000F7B5170001938A686D
:105640000B6900900C00934200DA130022003B60CB
:1056500043321278002A01D001333B6023689B0655
:1056600002D53B6802333B60062523681D401ED0EF
:10567000230043331B785A1E9341226892061CD59F
:105680003020E1184331087021005A1C4531097857
:10569000A2184332023311700FE0220001231932A5
:1056A00001990098089EB047431C0ED00135E3686D
:1056B0003A689B1A9D42F0DBDAE7220001994332F7
:1056C0000098089DA847431C02D10120404220E0D9
:1056D00006232068E1683A6803400025042B03D1C3
:1056E0008D1AEB43DB171D40A3682269934201DD4D
:1056F0009B1AED180027BD420AD0220001231A325E
:1057000001990098089EB047431CDED00137F2E7AC
:105710000020FEBDF0B58BB006920A00433207931D
:10572000059004920A7E0C00109B6E2A00D1ABE01B
:1057300011D8632A22D009D8002A00D1B5E0582A0E
:1057400000D0C5E045310A70814A4FE0642A1DD07F
:10575000692A1BD0BCE0732A00D1AAE009D86F2ABD
:1057600029D0702A00D0B3E0202209680A432260C1
:1057700037E0752A1FD0782A33D0A9E00E001A68C6
:105780004236111D196013683370A4E021681A684D
:10579000080606D4490604D5111D19600023D55EFC
:1057A00002E0111D19601568002D3BDA2D23049AC3
:1057B0006D42137036E021681A68080606D449065F
:1057C00004D51568111D1960ADB202E0111D1960F4
:1057D00015685F4B227E039308276F2A1DD00A2786
:1057E0001BE022007821453211705A4A1968039251
:1057F000081D226818600D68100602D4500600D5F6
:10580000ADB2D30702D520231A4322601027002D02
:1058100003D1202322689A432260230000224333CD
:105820001A7002E00A274A4B03936368A360002BB7
:1058300009DB0422216891432160002D05D1049EDB
:10584000002B11D07BE0002D79D0049E2800390078
:10585000FFF764FB039B013E5B5C2800337039005B
:10586000FFF7D6FA051EF1D1082F09D12368DB070F
:1058700006D563682269934202DC3023013E33700F
:10588000049B9B1B23612BE009681A68080607D458
:10589000490605D5111D19601368A28A1A8004E013
:1058A000111D1960136862691A600023049E236148
:1058B00016E01A68111D1960166800216268300030
:1058C00000F064FC002801D0801B6060636803E086
:1058D000260042363270012323610023049A13709C
:1058E000079B09AA00932100069B0598FFF7A4FED9
:1058F000431C02D10120404227E02369320006996F
:105900000598079DA847431CF4D0236800259B07F2
:105910000FD4099BE068984217DA180015E02200BE
:105920000123193206990598079EB047431CE1D020
:105930000135E368099A9B1A9D42F0DBE9E72600EE
:10594000039B42361B7833708EE70BB0F0BDC04628
:105950002572000036720000154B10B51C68A36B51
:10596000002B15D11820FFF761FC124BA0630380B8
:10597000114B01224380114B8380114BC380114B8B
:105980000381052343810633838100230261436140
:10599000A46B0D4A206961690C4BFFF7AFFB012234
:1059A000002380185941206161614800400810BD02
:1059B000580100200E330000CDABFFFF3412000071
:1059C0006DE6FFFFECDEFFFF2D7F954C2DF4515867
:1059D000002370B5064C05000800236000F0C8FEE7
:1059E000431C03D12368002B00D02B6070BDC04640
:1059F000002000200CB430B5164B9DB00C1E1D6865
:105A000004DA8B2301202B6040421DE0822302A98F
:105A10009B008B810023029008619C4200D0631E92
:105A20008B604B6101235B42CB81209A21AB280024
:105A3000019300F053FC431C01DA8B232B60002CF4
:105A400002D00023029A13701DB030BC08BC02B013
:105A50001847C046580100200EB410B59DB002A9E9
:105A6000029008610B48822488604861012040420E
:105A70001FABC881084804CBA400006801938C8147
:105A800000F02CFC0023029A13701DB010BC08BC5F
:105A900003B01847FFFFFF7F5801002002780B7802
:105AA000002A03D0013001319A42F7D0D01A704752
:105AB000031C0A7801311A700133002AF9D17047AA
:105AC0000023C25C0133002AFBD1581E704703003B
:105AD00030B5002A0DD00C7801335D1E013A2C70D0
:105AE0000131002CF5D19A189A4202D01C70013372
:105AF000FAE730BDF0B51E00454B87B01B68019238
:105B0000029308220B00059003911C7802995D1CFA
:105B100009194878104001D02B00F6E72D2C04D14C
:105B20009D1C5C780123009304E000902B2C01D194
:105B30005C789D1C002E02D0102E0AD162E0302C21
:105B40005ED120222B789343582B54D110266C78A9
:105B50000235009F31007B1E9F412E4BFF183800FD
:105B6000FFF7DCF9380004913100FFF751F9002309
:105B70000322070094461800029A12195178042251
:105B8000114201D0303C07E06246114017D0372265
:105B9000012900D02032A41AA64210DD5A1C0BD0D5
:105BA000B84207D802D1049B9C4203DC7043012316
:105BB000201801E001235B422C780135DCE75A1CF8
:105BC0000BD10098059A431E9841124BC01822230E
:105BD0001360019B002B0AD117E0009A002A00D025
:105BE0004042019A002A10D0039A002B00D06A1E6E
:105BF000019B1A6009E03024002EAAD10826A8E7EC
:105C00000A26A6E7302C9CD0A3E707B0F0BDC0461B
:105C10005C010020FFFFFF7F10B513000A000100A8
:105C200002480068FFF766FF10BDC046580100201B
:105C3000F8B505000F001400002804D08369002B7C
:105C400001D100F0BDF9234B9C4201D16C6808E002
:105C5000214B9C4201D1AC6803E0204B9C4200D117
:105C6000EC68A369A360A3891B070AD52369002BED
:105C700007D023682269FEB2981A636998420FDB45
:105C800008E02100280000F02BF80028F1D00120C6
:105C900040421DE02100280000F024F90028F6D140
:105CA000A3680130013BA36023685A1C22601F7067
:105CB0006369984205D0A3893000DB0708D50A2E16
:105CC00006D12100280000F00DF90028DFD13000B6
:105CD000F8BDC04648730000687300008873000078
:105CE000354B70B51D6806000C00002D05D0AB6962
:105CF000002B02D1280000F063F9304B9C4201D107
:105D00006C6808E02E4B9C4201D1AC6803E02D4B3F
:105D10009C4200D1EC68A3899AB2110723D4D10622
:105D200007D409220120326037321343A381404255
:105D300040E0530713D5616B002908D0230044339A
:105D4000994202D03000FFF797FA002363632422C0
:105D5000A3899343A38100236360236923600822FE
:105D6000A3891343A3812369002B0BD1A023A2890C
:105D70009B00134080229200934203D02100300008
:105D800000F0B2F90123A289134005D00023A360DB
:105D900063695B42A36103E0910700D46369A36078
:105DA00000202369834205D1130603D540231A43FB
:105DB000A281013870BDC046580100204873000020
:105DC000687300008873000010B5062000F0AEFB79
:105DD000012000F0E3FC0000F7B58A8905000C0003
:105DE00013075AD44B68002B02DC0B6C002B19DD17
:105DF000E76A002F16D000232E682B6080235B01FA
:105E00001A4001D0606D14E00123216A2800B847D0
:105E1000431C0ED12B68002B0BD01D2B01D0162B51
:105E200002D12E6000205AE04022A3891343A381AF
:105E300055E0A3895B0706D56368C01A636B002B26
:105E400001D0236CC01A00230200216A2800E76AEF
:105E5000B847A389421C06D129681D293AD8204A8F
:105E6000CA40D20736D50022626022692260DB0474
:105E700005D5431C02D12B68002B00D16065616BF6
:105E80002E600029CED023004433994202D028004E
:105E9000FFF7F2F90020606321E00F69002FC1D005
:105EA0000B680F60DB1B01930023920700D14B6945
:105EB000A36003E0019B3F181B1A0193019B002B79
:105EC000B0DD019B3A00216A2800A66AB04700288D
:105ED000F0DCA389402201201343A3814042FEBD90
:105EE000010040200B6970B505000C00002B01D1AA
:105EF00000201CE0002804D08369002B01D100F0B1
:105F00005FF80B4B9C4201D16C6808E0094B9C4246
:105F100001D1AC6803E0084B9C4200D1EC680C2234
:105F2000A35E002BE4D021002800FFF755FF70BDD1
:105F300048730000687300008873000010B50249C0
:105F400000F0B0F810BDC046E55E0000002310B5BB
:105F5000040003604360836081814366C281036102
:105F600043618361190008225C30FFF77CF9054B1F
:105F700024626362044BA362044BE362044B236319
:105F800010BDC0466D65000095650000CD65000040
:105F9000F965000070B568254B1E5D430E002900B1
:105FA0007431FFF7AFF9041E08D000212A00016008
:105FB00046600C30A0606832FFF755F9200070BDD4
:105FC000836913B50400002B28D18364C36403657F
:105FD000134B144A1B6882620193984201D101233A
:105FE0008361200000F020F86060200000F01CF8C1
:105FF000A060200000F018F80022E0600421606832
:10600000FFF7A4FF01220921A068FFF79FFF0222EA
:106010001221E068FFF79AFF0123A36113BDC04678
:10602000107200003D5F0000F8B51D4B06001D68B2
:10603000AB69002B02D12800FFF7C2FF4835AC68DE
:106040006B68013B05D40C22A75E002F10D068348A
:10605000F7E72B68002B01D02D68F0E70421300012
:10606000FFF798FF28600028F6D10C23336016E074
:10607000012320005B42E3810233A381676627602E
:10608000A760676027616761A7615C3008223900FB
:10609000FFF7E9F820006763A763A764E764F8BD2A
:1060A00010720000F7B50400070000260191483483
:1060B000002C16D06368A5680093009B013B0093F9
:1060C0000DD4AB89012B08D90E22AB5E013304D06D
:1060D00029003800019B984706436835EDE724689E
:1060E000E6E73000FEBD0000F0B58B8991B00600F8
:1060F0000C009B0726D40E23C95E002904DA8023F6
:10610000A5891D4010D10CE001AA00F0A1FA0028D9
:10611000F5DBF023029D1B021D401A4BED186B426C
:106120005D418027FF0001E0002540273900300055
:10613000FFF7E8F800280CD1A3899A051FD40222A2
:106140001343A38123004733236023610123636149
:1061500015E080220C4BB362A38920601343A38116
:1061600020616761002D0AD00E23E15E300000F04F
:1061700081FA002803D00122A3891343A38111B01F
:10618000F0BDC04600E0FFFF3D5F0000C9B28218CD
:10619000904204D003788B4202D00130F8E700200F
:1061A000704710B5884202D98B18984201D300235A
:1061B00005E09B1A013A08D3995C8154FAE79342AF
:1061C00003D0CC5CC4540133F9E710BDF8B5060028
:1061D0000C001500002904D11100FFF793F804000A
:1061E00018E0002A03D1FFF747F82C0012E000F076
:1061F00067FA85420ED929003000FFF783F8071EA1
:1062000007D021002A00FFF725F821003000FFF712
:1062100033F83C002000F8BDF0B58E6885B007006B
:106220000C00039201939E4243D890238A89DB009D
:106230001A423ED003250969236801985B1A02932C
:1062400063695D43EB0F5D19029B6D1001331B18F1
:10625000AB4200D91D00530510D529003800FFF7C7
:1062600051F8061E14D0029A2169FEF7F3FFA289A5
:10627000194B134080221343A38112E02A003800F7
:10628000FFF7A4FF061E0CD121693800FEF7F4FFCA
:106290000C23402201203B60A38940421343A38189
:1062A00017E0029B2661F61826606561019EED1AD3
:1062B000A560019BB34200D21E0032000399206802
:1062C000FFF76FFF0020A3689B1BA36023689E1944
:1062D000266005B0F0BDC0467FFBFFFFF0B59FB064
:1062E000029005938B890F0016001B0610D50B69D1
:1062F000002B0DD14021FFF705F8386038610028E8
:1063000004D10C23029A01381360D8E040237B614A
:10631000002306AD6B6120336B761033AB7634000F
:106320002378002B03D1A31B049312D003E0252B69
:10633000F9D00134F4E7A31B320039000298FFF7CB
:106340006BFF431C00D1B4E06A69049B944663442C
:106350006B612378002B00D1ABE001220023524275
:106360006A6002A95432521801342B60EB60AB60B2
:106370001370AB65534E217805223000FFF706FFFE
:10638000002807D00123801B83402A68013413436F
:106390002B60EFE72B68DA0604D55322202102A8F0
:1063A000121811701A0704D553222B2102A81218B3
:1063B000117022782A2A03D0099B00200A210EE0BE
:1063C000059A111D12680591002A01DB099204E06B
:1063D0005242EA60022213432B6001340BE0227820
:1063E000303A092A04D84B4301349B180120F6E7C0
:1063F000002800D0099323782E2B1ED163782A2BF6
:106400000AD1059B02341A1D1B680592002B01DA84
:1064100001235B42079310E000230A201A00013495
:106420006B6021783039092904D84243013452186D
:106430000123F6E7002B00D00792234E2178032298
:106440003000FFF7A3FE002806D04023801B8340C6
:106450002A68013413432B60217806221B48661CEE
:106460002976FFF793FE002812D0194B002B06D196
:106470000722059B073393430833059314E005ABCC
:1064800000933A00134B2900029800E000BF07E098
:1064900005AB00933A000F4B29000298FFF73AF939
:1064A0000390039B013304D06B69039A9B186B61C3
:1064B00035E7BB890B985B0601D5012040421FB030
:1064C000F0BDC046147200001A7200001E72000077
:1064D000000000001962000070B504000D1E1F2DA1
:1064E00004D916230360012040421EE0426C002ABA
:1064F00004D08B00D2181368002B08D1200000F0C4
:1065000031F82A000100200000F01AF80DE0002008
:10651000012B0AD0591C03D117332360013004E04A
:106520000024280014609847200070BD10B5034B6C
:1065300001001868FFF7D0FF10BDC04658010020C9
:10654000002370B5064C050008001100236000F020
:10655000F7F8431C03D12368002B00D02B6070BDDB
:106560000020002010B500F0DBF810BD70B50C0065
:106570000E25495F00F0B0F8002803DB636D1B189F
:10658000636503E0A289024B1340A38170BDC0463E
:10659000FFEFFFFFF8B51F008B8905000C00160008
:1065A000DB0505D50E23C95E0022022300F074F836
:1065B000A289054B28001340A38132000E23E15E1F
:1065C0003B0000F01FF8F8BDFFEFFFFF70B50C00B7
:1065D0000E25495F00F060F8A389421C03D1054AEB
:1065E0001340A38104E0802252011343A38160651C
:1065F00070BDC046FFEFFFFF10B50E23C95E00F06F
:1066000015F810BD70B50500080011000022064CF9
:1066100022601A0000F0BAF8431C03D12368002B53
:1066200000D02B6070BDC04600200020002370B554
:10663000064C05000800236000F062F8431C03D1FB
:106640002368002B00D02B6070BDC04600200020C6
:10665000002370B5064C050008001100236000F00F
:1066600057F8431C03D12368002B00D02B6070BD6A
:1066700000200020002370B5064C050008002360B0
:1066800000F056F8431C03D12368002B00D02B6088
:1066900070BDC0460020002070B505000800110044
:1066A0000022064C22601A0000F052F8431C03D16D
:1066B0002368002B00D02B6070BDC0460020002056
:1066C0000B1F1A68101F002A04DA891804390B6896
:1066D000D01804387047000070B50500080011009C
:1066E0000022064C22601A0000F03AF8431C03D145
:1066F0002368002B00D02B6070BDC0460020002016
:1067000058220120014B40421A60704700200020AF
:1067100058220120014B40421A607047002000209F
:1067200058220120014B40421A607047002000208F
:106730005822024B00201A607047C04600200020FB
:1067400058220120014B40421A607047002000206F
:1067500058220120014B40421A607047002000205F
:1067600058220120014B40421A607047002000204F
:10677000044A1368002B03D01818106018007047E3
:10678000014BF9E7A8100020082000205822012022
:10679000014B40421A60704700200020FEE7C046CF
:1067A000F8B5C046F8BC08BC9E467047F8B5C04670
:1067B000F8BC08BC9E467047F6060000880600003C
:1067C000060700003C07000078070000B207000041
:1067D000EE07000016080000540800009A080000A8
:1067E000F60800003A090000A0090000EC090000CA
:1067F000140A00004E0A0000980A0000C00A0000B7
:10680000F80A0000300B00006C0B0000F20B0000D7
:10681000BA0C0000480D0000A60D0000E80D0000B5
:106820000A0E0000120E0000F40E0000F606000032
:10683000F6060000F6060000F6060000400F000015
:10684000AA0F0000141000005E100000C01000002D
:1068500046110000CE1100001C120000661200005C
:10686000AC120000F8120000441300009013000066
:10687000DE1300003414000072140000DE14000067
:106880000E1500005A150000A6150000F2150000B4
:106890002C16000078160000F6060000F606000030
:1068A000F6060000F6060000C4160000F41600000C
:1068B000241700005017000080170000AC170000DC
:1068C000F6060000F6060000F6060000F6060000D8
:1068D000E41700002C18000078180000A818000029
:1068E000D4180000021900004C190000F606000040
:1068F000F6060000F60600007A190000AA1900004A
:10690000DA1900000A1A0000361A0000661A0000A0
:10691000921A0000BC1A0000E61A0000161B0000C4
:10692000461B0000881B0000B41B0000E41B000095
:10693000101C0000F6060000F6060000F606000037
:10694000F6060000F6060000401C00006C1C00006B
:10695000981C0000C41C0000F01C0000281D000052
:10696000601D0000981D0000D01D0000FC1D0000EF
:106970002A1E00005A1E0000F6060000F60600005F
:10698000F6060000F6060000F6060000F606000017
:10699000F6060000F6060000F6060000F606000007
:1069A000F6060000F6060000F6060000F6060000F7
:1069B000881E0000B61E000066616C73650074726C
:1069C0007565006C697374206F6620256420697496
:1069D000656D73006F626A656374206F6620636C17
:1069E0006173733A20256400537461636B20756E84
:1069F000646572666C6F77000D0A564D2050616EAB
:106A000069633A2025730D0A00496E7375666669DD
:106A10006369656E74206D656D6F727920666F7243
:106A2000204D6963726F426C6F636B73206F626A93
:106A3000656374206865617000496E737566666988
:106A40006369656E74206D656D6F727920666F7213
:106A5000204D6963726F426C6F636B732073746156
:106A6000636B00626164206F626A656374206174A5
:106A700020256C640A0025783A20256420776F72FF
:106A800064732C20636C61737349442025640A008D
:106A90004865616465723A2025780A0009307825D6
:106AA000782C0A0025642025642025642025640AAA
:106AB00000426164207265636F726420666F756E58
:106AC0006420647572696E6720696E697469616CAF
:106AD000697A6174696F6E210A004E6F7420656E69
:106AE0006F75676820726F6F6D206576656E2061C7
:106AF0006674657220636F6D70616374696F6E0A8E
:106B000000526573746F72696E6720256420736329
:106B100072697074732E2E2E0053746172746564E2
:106B2000002D2D2D2D2D0A0050657273697374652B
:106B30006E74204D656D6F727920546573740A0A06
:106B4000000A496E697469616C697A696E67204DE3
:106B5000656D6F72790A004D656D6F727920696E8F
:106B600074697469616C697A65643B2077726974D1
:106B7000696E67207265636F7264732E2E2E0A0031
:106B80005265636F7264206174206F66667365740A
:106B90002025643A2025642025642025642025646E
:106BA0002028256420776F726473290A0046696E75
:106BB000616C3A2063757272656E7420256420756D
:106BC00073656420256420633020256420633120B0
:106BD00025640A004E6F2066726565207461736BD0
:106BE00020656E74726965730057656C636F6D65BF
:106BF00020746F204D6963726F426C6F636B7321F9
:106C0000004D656D6F727920636C65617265642EED
:106C100000416C6C207461736B732073746F7070BF
:106C20006564007630343800202573202573000019
:106C300007000000030000006D6963726F3A62692B
:106C40007400696F00686173546F6E6500706C61E9
:106C500079546F6E6500686173536572766F007367
:106C60006574536572766F0000000000010000003B
:106C70000200000003000000040000000A00000001
:106C80006E65740068617357694669007374617258
:106C900074576946690073746F7057694669007765
:106CA000696669537461747573006D794950416404
:106CB0006472657373007468696E674465736372A8
:106CC000697074696F6E00636C6561725468696E97
:106CD000674465736372697074696F6E0061707088
:106CE000656E64546F5468696E6744657363726956
:106CF0007074696F6E001A1B1C03040607090A17DB
:106D000018191A1B1C03040607090A1718196469C5
:106D100073706C6179006C696768744C6576656C3A
:106D20000000000000000000010000000200000060
:106D30000300000004000000050000000600000041
:106D40000700000008000000090000000A00000021
:106D50000B0000000C0000000D0000000E00000001
:106D60000F000000100000001200000014000000DE
:106D700016000000180000001A0000001C000000AF
:106D80001E0000002000000023000000260000007C
:106D9000290000002C0000002F000000320000003D
:106DA000360000003A0000003E00000042000000F3
:106DB000460000004B00000050000000550000009D
:106DC0005A00000061000000680000006F00000031
:106DD000760000007D000000840000008B000000B1
:106DE0009200000099000000A0000000A700000031
:106DF000AE000000B5000000BC000000C3000000B1
:106E0000CA000000D1000000D8000000DF00000030
:106E1000E6000000ED000000F4000000FB000000B0
:106E2000FF000000000000000008080800080A4AEF
:106E30004000000A5FEA5FEA0ED92ED36E19324491
:106E400089330C924C924D08080000000488080811
:106E5000040804848488000A448A4000048EC480A4
:106E6000000000048800000EC000000000080001BF
:106E7000224488100C9252524C048C84848E1C82C2
:106E80004C901E1EC244924C06CA525FE21FF01E76
:106E9000C13E02448ED12E1FE24488100ED12ED165
:106EA0002E0ED12EC488000800080000048004883B
:106EB0000244880482000EC00EC008048244880E7A
:106EC000D126C0040ED135B36C0C925ED2521C9206
:106ED0005C925C0ED010100E1C9252525C1ED01CA4
:106EE000901E1ED01C90100ED013712E12525ED226
:106EF000521C8808081C1FE242524C1254981492EB
:106F0000101010101E113B75B131113935B3710CD1
:106F10009252524C1C925C90100C92524C861C92D5
:106F20005C92510ED00C825C1FE484848412525215
:106F3000524C1131312A44113135BB7112524C92ED
:106F400052112A4484841EC488101E0EC808080EDC
:106F500010080482410EC242424E048A40000000E2
:106F60000000001F0804800000000ED2524F1010D5
:106F70001C925C000ED0100E02424ED24E0C925C5F
:106F8000900E06C81C88080ED24EC24C10101C92DF
:106F9000520800080808024002424C10149814924B
:106FA0000808080806001B75B131001C92525200F7
:106FB0000C92524C001C925C90000ED24EC2000EFD
:106FC000D010100006C8049808080EC80700125216
:106FD000524F0011312A4400113135BB00124C8C44
:106FE0009200112A4498001EC4881E06C48C848610
:106FF000080808080818080C881800000C8360733B
:10700000656E736F72730074656D7065726174750F
:1070100072650074696C74580074696C74590074FA
:10702000696C745A00746F756368526561640074AA
:10703000667400656E61626C65446973706C617939
:1070400000736574506978656C00535049436C61F6
:1070500073733A3A535049436C617373284E5246E6
:107060005F5350495F547970652A2C2075696E749E
:10707000385F742C2075696E74385F742C207569C4
:107080006E74385F742900705F73706920213D2031
:107090004E554C4C002F55736572732F6A6F686E96
:1070A0006D616C6F6E65792F4C6962726172792FB8
:1070B00041726475696E6F31352F7061636B616702
:1070C00065732F73616E646565706D697374727931
:1070D0002F68617264776172652F6E5246352F306A
:1070E0002E362E302F6C69627261726965732F5370
:1070F00050492F5350492E6370700000000000006B
:10710000000000001F420000E54100000B420000AB
:107110001542000045420000094200000300000043
:107120000200000001000000040000000500000053
:10713000110000000C0000000B0000001200000015
:107140000A000000060000001A0000001400000001
:1071500017000000160000001500000010000000DD
:10716000FFFFFFFFFFFFFFFF000000001E00000009
:1071700019000000180000000700000008000000CF
:10718000090000000D0000000E0000000F000000CC
:107190001C0000001B0000001D0000001300000088
:1071A0000000000000000000014A0000214900002A
:1071B000714A0000854A00007B4A0000FF49000038
:1071C000F3490000914A00001D4A0000EF49000009
:1071D0002C2066756E6374696F6E3A20006173735C
:1071E000657274696F6E2022257322206661696C56
:1071F00065643A2066696C6520222573222C206C18
:10720000696E65202564257325730A00430000001C
:10721000F8000020232D302B2000686C4C006566A0
:1072200067454647003031323334353637383941D7
:1072300042434445460030313233343536373839ED
:1072400061626364656600002020202020202020E9
:107250002028282828282020202020202020202006
:107260002020202020202020881010101010101026
:10727000101010101010101004040404040404046E
:1072800004041010101010101041414141414101FF
:1072900001010101010101010101010101010101DE
:1072A00001010110101010101042424242424202ED
:1072B00002020202020202020202020202020202AE
:1072C0000202021010101020000000000000000058
:1072D00000000000000000000000000000000000AE
:1072E000000000000000000000000000000000009E
:1072F000000000000000000000000000000000008E
:10730000000000000000000000000000000000007D
:10731000000000000000000000000000000000006D
:10732000000000000000000000000000000000005D
:10733000000000000000000000000000000000004D
:10734000000000000000000000000000000000003D
:10735000000000000000000000000000000000002D
:10736000000000000000000000000000000000001D
:10737000000000000000000000000000000000000D
:1073800000000000000000000000000000000000FD
:1073900000000000000000000000000000000000ED
:0C73A000000000000000000000000000E1
:0873AC00C88DFF7F0100000005
:1073B400FFFFFFFF456C0000FD3100004D6C000035
:1073C400F9310000566C0000013200005F6C0000CF
:1073D40005320000846C0000B53400008C6C0000A1
:1073E400D9340000966C0000E33400009F6C000068
:1073F400ED340000AA6C0000F7340000B66C000005
:10740400C3340000C76C0000CD340000DD6C000004
:10741400B9340000166D0000193500001800000092
:10742400FF00000007700000293D000013700000F9
:10743400F13F000019700000014000001F700000BF
:1074440011400000257000005D3D00003370000015
:1074540025400000417000002140000003000000AE
:1074640002000000080000000A000000FFFFFFFF08
:107474000000000001000000000002000100000004
:10748400FFFFFFFF000000000200000000000400F6
:1074940002000000FFFFFFFF0000000003000000E7
:1074A4000000080003000000000000004873000012
:1074B40068730000887300000000000000000000F2
:1074C40000000000000000000C720000000000003A
:1074D40000000000000000000000000000000000A8
:1074E4000000000000000000000000000000000098
:1074F4000000000000000000000000000000000088
:107504000000000000000000F800002047720000A6
:1075140039010000B541000099440000F54C000019
:087524000D0100000000000051
:04000003000044B104
:00000001FF
